:2000000002002E02713FFFFFFFFFFFFFFFFFFFFFFFFFFFFFFFFFFFFFFFFFFFFFFFFFFFFF18
:20002000FFFFFFFFFFFFFFFFFFFFFF02715B7581AB90F8008583A0124A3A53B1FEEC4D60FB
:200040005178AB7600D8FC90FA47AE83AF8290F8B812009B6005E4F0A380F690F800A982BD
:2000600090F800A882E899500576000880F79000F91200A49000FD1200A49001011200A439
:200080009001051200C290010B1200C29001111200C275D000124ECB020117EF658270033D
:2000A000EE658322E493F8740193F9740293FE740393F5828E83E869700122E493F6A30843
:2000C00080F4E493FC740193FD740293FE740393FF740493F8740593F582888312009B7076
:2000E0000122E493A3A883A9828C838D82F0A3AC83AD828883898280E3212114A521211494
:20010000A5A8AC14A5F80014A914A9FA4714AD14A9FA4B274F274F80FECCC0E01201452C5D
:200120008002D0F030F00920F303F68010F7800D30F10920F303F28004F38001F020F40402
:20014000FCD0E0CC22BF000775F001EDF8E622BF010975F0048D828E83E02275F002EDF84C
:20016000E222EEF8EFF902016DECF8EDF9E88BF0A4C98AF0A429F9E88AF0A4F8E5F029F96E
:200180004822EEF8EFF902019AECF8EDF902019AECF8EDF9EBC9FBEAC8FAEB335008E4C3E1
:2001A0009AFAE49BFBD392F0E930E709B2F0C3E498F8E499F91201FD30F008C3E498F8E431
:2001C00099F94822ECF8EDF90201D5ECF8EDF9EBC9FBEAC8FA89F012019A20F706EAF8EB4C
:2001E000F94822C3E49AF8E49BF94822ECF8EDF90201FDECF8EDF9EBC9FBEAC8FAE94B70EE
:2002000010E8C0F08AF084F8AAF0D0F079007B0022ECC0E0EDC0E0EEC0E07D007E007C10A2
:20022000C3E833F8E933F9ED33FDEE33FEED9AEE9B4005FEED9AFD08DCE6EDFAEEFBD0E076
:20024000FED0E0FDD0E0FCE8492230E01B20E30C08E625F0F6F5F018E63CF62209E725F085
:20026000F7F5F019E73CF72230E211C083A3E025F0F5F0F01582D083E03CF02220E30C084B
:20028000E225F0F2F5F018E23CF22209E325F0F3F5F019E33CF3227900900001F5F0E9CC7C
:2002A000F912120A800012024AC9FCE5F022F5F0EBCCFB1211E7800F7B00900001F5F0EB71
:2002C000CCFB12120A800012024ACBFCE5F0227D00900001F5F0EDCCFD1211B48000120279
:2002E0004ACDFCE5F022ECF8EDF9EEFAEFFBEF4E4D4B4A49700DE88CF0A4FCADF07E007FD5
:20030000004D22C082ECF58288F0A4C0E0E8C5F0CDC0E0A42DFDE435F0CEFC8582F0E9A4DE
:200320002DFDEE35F0FEE433CF88F0A42FFFE98CF0A42FFFEAD0F0C0F0A42FFFEB8582F00D
:20034000A42FFFD0F0E9A42EFEEF35F0FFEA8582F0A42EFEEF35F0FF8CF0E8A42EFEEF3523
:20036000F0FFD0E0D082FC4E4D4F22EFCBFFEECAFEEDC9FDECC8FC2212036BEB4A4E4F70CE
:2003800017ECFAEDFB1201F7F5F0E8FCE9FDEAF8EBF9E4FAFBE5F022C082C08375F0208B94
:2003A000828883E4FBCFC0E0E4CACEC0E0E4C9CDC0E0C3EC33FCA881E633F618E633F618D7
:2003C000E633F6EB33FBE933F9EA33FAEF33FFEB9583E99DEA9EEF9582400CFFEB9583FB48
:2003E000E99DF9EA9EFA0CD5F0C8D0E0FDD0E0FEEBF8D0E0CFFBECD083D0824D4E4F2212FC
:20040000036B12037BEBFFEAFEE9FDE8FC80EC12036BEB33500EE4C398F8E499F9E49AFAB5
:20042000E49BFBD3EF30E708B3C0D01204518002C0D012037BD0F020F70122F5F0120451CF
:20044000E5F02212036BEFC0E012041212040580E4E4C39CFCE49DFDE49EFEE49FFF4E4D95
:200460004C22ECF4FCEDF4FDEEF4FEEFF4FF4E4D4C22C083F5F0C3EC98F583ED994283EE69
:200480009A428320F010C082EB6480F582EF64809582D0828002EF9B82F130F2054583703B
:2004A00001D3D08330F301B3E4332288F005F0800EEFA2E713FFEE13FEED13FDEC13FCD5B4
:2004C000F0EFEF4E4D4C2288F005F0800DC3EF13FFEE13FEED13FDEC13FCD5F0F0EF4E4D51
:2004E0004C2288F005F0800DC3EC33FCED33FDEE33FEEF33FFD5F0F0EF4E4D4C228CF0052B
:20050000F0800DC3E833F8E933F9EA33FAEB33FBD5F0F0EB4A494822ECF8EDF9EEFAEFFB0A
:20052000EC28FCED39FDEE3AFEEF3BFF4E4D4C22C3EC98FCED99FDEE9AFEEF9BFF4E4D4C74
:2005400022EC58FCED59FDEE5AFEEF5BFF4E4D4C22EC48FCED49FDEE4AFEEF4BFF4E4D4CA5
:2005600022EC68FCED69FDEE6AFEEF6BFF4E4D4C22080808E64CFCF618E64DFDF618E64E38
:20058000FEF618E64FFFF64E4D4C22080808C3E496FCF618E496FDF618E496FEF618E49638
:2005A000FFF64E4D4C2275F091EBC0E0EAC0E0E9C0E0E8C0E0EDF9EEFAEFFBE6FF08E6FE98
:2005C00008E6FD08E6CCC830F310CCC0E0CCCDC0E0CDCEC0E0CECFC0E0CFC0E00205EAE816
:2005E00014600104F9FAFB020520C0F0E5F0C4540F75F005A49005F973120520804912059B
:200600003080441202EE803F120412803A12037B80351204468030120402802B1204AB80EE
:20062000261204C780211204E2801C12054180171205518012120561800D1205DF80081204
:2006400004518003120462D0F0FB30F010D0E0F8ECF618EDF618EEF618EFF6802E30F21DF4
:20066000D083D082EFF0A3EEF0A3EDF0A3ECF0E58224FDF582E58334FFF583800ED0E0F82E
:20068000ECF218EDF218EEF218EFF230F310D0E0FFD0E0FED0E0FDD0E0FC4D4E4FFBD0E016
:2006A000F8D0E0F9D0E0FAD0E0CB2275F044800375F0F4EBC0E0EAC0E0E9C0E0E8C0E0ECBB
:2006C000F8EDF9EEFAEFFBE0FFA3E0FEA3E0FDA3E0FC30F30CECC0E0EDC0E0EEC0E0EFC086
:2006E000E0E58224FDC0E0E58334FFC0E00205EAE4F8F90206FEECF8EDF9EEFAEFFBEF4E12
:20070000700122EB4A7005FFFCFDFE22120966947F40092B500C7F7F74FF80EC2B4003E4F1
:2007200080E5C0E0C0F0E849704EBA8009D0E0F9D0E0F8020828EC4D7018BE8008E8FCE97B
:20074000FDEAFE80E8E4FBFFEA8EF0A4F8E5F00207F2EA8CF0A4FFABF0EA8DF0A42BFBE4E1
:2007600035F0F8EA8EF0A428F8E435F00207F2EACEFAE9FDE8FC80DAEC4D7005BE80F080FA
:20078000BCEAC0E0EC88F0A4FFABF0ED88F0A42BFBE435F0FAEC89F0A42B4FFFE5F03AFAB4
:2007A000E433FB88F0EEA42AFAE5F03BFBED89F0A42AFAE5F03BFBE433F88CF0D0E0FCA4DA
:2007C0002AC5F03BFBE438F8EF6002D2F0AFF0ED8CF0A42BFBE5F038F8E433FAEE89F0A4EA
:2007E0002BFBE5F038F8E43AFAEC8EF0A428F8E5F03AF5F0FEE8FDEBFCD0E0F9D0E0F83049
:20080000F70608B80005802D1208418000EF3350178CF020F00260100CBC000C0DBD000861
:200820000EBE000408E8600DE933E813FFEE2313FE4F4D4C227F7F74FF8002E4FFFEFDFC7C
:2008400022C3EF33FFEC33FCED33FDEE33FE22C3EE13FEED13FDEC13FCEF135002D2E0FF5A
:2008600022C3E49CFCE49DFDE49EFEE49FFF22E4F8F9800FE4FCFDEFCBFFEECAFEEDC9FD12
:20088000ECC8FCEF4E60B4EB4A60AA120966EB947FCF40059F500680A2C39F5098FBE849F8
:2008A000700CEA94807007EBF8A9F0020828C0F07F00120957501EEB6002DB05D0F0020893
:2008C0003BC3120845EF33FFEC28FCED39FDEE3AFEE43FFFD3EBC0E075F0087403C0E07BC2
:2008E00000501CC3EC98FCED99FDEE9AFEEF9400FF500CEC28FCED39FDEE3AFEE43FFFEBFC
:2009000033FBEC33FCED33FDEE33FEEF33FFD5F012D0F0EBC0E0E5F0146012C0E075F008A7
:200920007B00EF20E0BDEED330E7D480B61209574E4D4CFBD0E0F4FCD0E0F4FDD0E0F4FE77
:20094000D0E0F8D0E0F9EB50030208286003020818EC5401020816C3EC98FCED99FDEE9AA2
:20096000FEEF9400FF22EAA2E7D2E7FAEB33FB13F5F0EEA2E7D2E7FEEF33FFC5F013A2E7FE
:2009800030E601B313C5F0C322E8FB7A80E4F9F88025ECFF7E80E4FDFC801CE4FCFDEFCB90
:2009A000FFEECAFEEDC9FDECC8FCEB4A7003EF4E22EB6480FB8007EB4A7003EF4E22EF4E83
:2009C000700BEBFFEAFEE9FDE8FC740122C3EC98ED99EE9AEBC2E7F5F0EFC2E795F0500E20
:2009E000600CEBCFFBEACEFAE9CDF9E8CCF8120966C0E0C0F07F00C39BFB605B9418600C4D
:200A0000401AD0E023F9D0E0F80208288AF0E9486003D2F0E4AFF0FAF9F8803BEB30E40DD1
:200A200089F0EA6003D2F0E4AFF0F9CAF8EB30E30D88F0EF6002D2F0AFF0E4CAC9F8EB540D
:200A4000076014FBC3EA13FAE913F9E813F8EF135002D2E0FFDBEDD0E0C0E030E734C3E46F
:200A60009FFFF5F0EC98FC42F0ED99FD42F0EE9AFE42F0D0E0F9D0E0F8E5F0700122E9230F
:200A8000F9EE30E70302080DD80302083B12084180F0EC28FCED39FDEE3AFED0E023F9D05E
:200AA000E0F8400302080D12085008B8000302083502080DEF4E7003FDFC22EEA2E7D2E786
:200AC000FEE4CF3392D5C3947F500302083BF5F0941F40056011020835F404F5F0EF54FEB2
:200AE000FF12084FD5F0F6EFCCCDCECF30D503120861EE020831E4FEFF8011ED3395E0FEFD
:200B0000FFEF30E707D2D51208618002C2D5EF4E4D4C70012275F096EF700EEE20E71C1597
:200B2000F012084130E7F88012EF05F0C313FFEE13FEED13FDEC13FCEF70EFA2D5E5F0136C
:200B4000FFEE92E7FE440122E93395E0FAFBEB30E711D2D5C3E498F8E499F9E49AFAE49BE6
:200B6000FB8002C2D5EB4A494870012275F096EB7018EA20E72615F0C3EB33FBE833F8E9A6
:200B800033F9EA33FA30E7EE8012EB05F0C313FBEA13FAE913F9E813F8EB70EFA2D5E5F055
:200BA00013FBEA92E7FA4401227800790080047C007D00F5F0C3EF20E706EB30E714803487
:200BC000EB20E704F4D3802C30F10363F00CEB547FFBEF4E7002FCFDEB4A7002F8F9EC98AC
:200BE000A8F0F5F0ED9942F0EE9A42F0EF547F9B45F088F082F130F2037001D330F301B349
:200C0000E4332275F014800375F054EBC0E0EAC0E0E9C0E0E8C0E0E0FBA3E0FAA3E0F9A349
:200C2000E0F830F30CE8C0E0E9C0E0EAC0E0EBC0E0E58224FDC0E0E58334FFC0E0804175EE
:200C4000F001800E75F021800975F031800475F049FCEBC0E0EAC0E0E9C0E0E8C0E080009C
:200C6000E6FB08E6FA08E6F908E6C830F310C8C0E0C8C9C0E0C9CAC0E0CACBC0E0CBC0E06F
:200C8000C0F0E5F0C4540F75F005A475829275830C731209B7803A12099E80351206FE800A
:200CA00030120877802B1209928026120D3180211209B7801C1209AA80171206FE80121200
:200CC0000883800D1209898008EF4E6004EFB2E7FFD0F0FB30F010D0E0F8ECF618EDF61820
:200CE000EEF618EFF6802E30F21DD083D082EFF0A3EEF0A3EDF0A3ECF0E58224FDF582E53E
:200D00008334FFF583800ED0E0F8ECF218EDF218EEF218EFF230F30CD0E0FFD0E0FED0E06D
:200D2000FDD0E0FCD0E0F8D0E0F9D0E0FAD0E0CB22E8FCE9FDEAFEEBFF4E6004EFB2E7FF9D
:200D400022D083D082F5F0C3E493A3C5F095F0C0E0C3D0F0E493A395F04012A3A3C3E5F0DE
:200D600033500205832582F58250020583740193C0E0E493C0E022D083D082F5F0E493701C
:200D8000097401937004A3A3800C74029365F06005A3A3A380E7740193C0E0E493C0E02208
:200DA00030F10678FF7CFF8007E84C7003E4FB22BB006CBF0017E8FCEDF8E7FAE6C39A7091
:200DC0006F30F003EA60660809DCEF8060BF011B8D828E83800209A3E7FAE0C39A705130DD
:200DE000F003EA6048D8EF80448000BF021A8D828E83800209A3E7FAE493C39A703230F0C3
:200E000003EA6029D8EE8025E8FCEDF8E7FAE2C39A701D30F003EA60140809DCEF800EBBD5
:200E2000015BBF002489828A83EDF9800BE4FB22FBE49400CB2209A3E0FAE7C39A70F1302E
:200E4000F003EA60E8D8EF80E4BF01358D828E83B8000280010CC9C582C9CAC583CAE0FB56
:200E6000A3C9C582C9CAC583CAE0C39B70C230F003EB60B9A3D8DFDCDD80B280008062805C
:200E800000BF023B8D828E83B8000280010CC9C582C9CAC583CAE0FBA3C9C582C9CAC583D1
:200EA000CAE493C39B701230F003EB6009A3D8DEDCDC80028009E4FB22FBE49400CB228994
:200EC000828A83EDF9E0FAE3C39A6003020EB930F006EA7003020EB609A3D8E9020EB6805B
:200EE00000BB0254BF001C89828A83EDF9800209A3E493FAE7C39A707830F003EA606FD889
:200F0000EE806BBF01348D828E83B8000280010CC9C582C9CAC583CAE493FBA3C9C582C9FA
:200F2000CAC583CAE0C39B704830F003EB603FA3D8DEDCDC803880598057BF023A8D828E21
:200F400083B8000280010CC9C582C9CAC583CAE493FBA3C9C582C9CAC583CAE493C39B7003
:200F60001030F003EB6007A3D8DDDCDB8000E4FB22FBE49400CB2289828A83EDF9E493FA8D
:200F8000E3C39A70EC30F003EA60E309A3D8EE80DDBF0019E8FCEDF8E3FAE6C39A70D23063
:200FA000F003EA60C90809DCEF80C38000BF011B8D828E83800209A3E3FAE0C39A70B230F7
:200FC000F003EA60A9D8EF80A58000BF021B8D828E83800209A3E3FA93C39A709430F003A1
:200FE000EA608BD8EF80878000E8FCEDF8E3FAE2C39A6003020F7130F006EA7003020F6E02
:201000000809DCE9020F6E121195800F1211B4800A1211E7800512120A800030E00720E37C
:2010200002E622E72230E10720E302E222E32230E202E022E493221211958000ADF01210D1
:201040005ACDC5F0CD2212120A80051211E78000ABF012105ACBC5F0CB2230E01020E306DB
:20106000E6F5F008E622E7F5F009E7192230E11020E306E2F5F008E222E3F5F009E31922B2
:2010800030E206E0F5F0A3E022E493F5F074019322121195804D1211E7800030E01520E311
:2010A00009E6FB08E6FA08E6F922E7FB09E7FA09E7F92230E11520E309E2FB08E2FA08E2A1
:2010C000F922E3FB09E3FA09E3F92230E209E0FBA3E0FAA3E0F922E493FB740193FA74022F
:2010E00093F92230E01720E309E6FF08E6FE08E6FD22E7FF09E7FE09E7FD19192230E117F4
:2011000020E309E2FF08E2FE08E2FD22E3FF09E3FE09E3FD19192230E209E0FFA3E0FEA3CA
:20112000E0FD22E493FF740193FE740293FD22121195800030E01E20E30CE6FF08E6FE08BE
:20114000E6FD08E6FC22E7FF09E7FE09E7FD09E7FC1919192230E11E20E30CE2FF08E2FE7F
:2011600008E2FD08E2FC22E3FF09E3FE09E3FD09E3FC1919192230E20CE0FFA3E0FEA3E075
:20118000FDA3E0FC22E493FF740193FE740293FD740393FC22BB0003740922BB01078982DC
:2011A0008A83740422BB020789828A83741022740A228000BB0007E92582F8740122BB0149
:2011C0000DE92582F582EA3583F583740422BB020DE92582F582EA3583F583741022E925A8
:2011E00082F87402228000BF0005EDF8740122BF01078D828E83740422BF02078D828E83B4
:20120000741022EDF87402228000BF0007ED2582F8740122BF010DED2582F582EE3583F5CF
:2012200083740422BF020DED2582F582EE3583F583741022ED2582F87402228000C0E0129E
:201240001195800EC0E01211E78007C0E012120A800030E00B20E304D0E0F622D0E0F72228
:2012600030E10B20E304D0E0F222D0E0F322D0E0F022C0E0EDC0E0121195800AC0E0EBC046
:20128000E01211E7800030E01420E308D0E0F6D0E008F622D0E0F7D0E009F7192230E11488
:2012A00020E308D0E0F2D0E008F222D0E0F3D0E009F31922D0E0F0D0E0A3F02212119580EE
:2012C0000030E01E20E30CEFF608EEF608EDF608ECF622EFF709EEF709EDF709ECF719192A
:2012E000192230E11E20E30CEFF208EEF208EDF208ECF222EFF309EEF309EDF309ECF31907
:20130000191922EFF0A3EEF0A3EDF0A3ECF02208A3E493F6D9F922E6FB08E6FA08E6F90438
:20132000F61870010622E6FF08E6FE08E6FD04F61870010622E0FFA3E0FEC083A3E0FD0478
:20134000F01582D0837003E004F022EEFAEDF904FD70010EEFFB22EEFAEDF91D70011EEF87
:20136000FB22D083D082EFC0E0EEC0E0EDC0E0ECC0E0E473D083D082EFC0E0EEC0E0EDC0AF
:20138000E0E473D083D082EBC0E0EAC0E0E9C0E0E8C0E0E473D083D082D0E0FCD0E0FDD026
:2013A000E0FED0E0FFE473D083D082D0E0F8D0E0F9D0E0FAD0E0FBE473EFF608EEF608EDE1
:2013C000F622EBF608EAF608E9F622EFF608EEF608EDF608ECF622EFF709EEF709EDF70991
:2013E000ECF722C0E0EBF608EAF608E9F608D0E0F6F822E6FF08E6FE08E6FD22E6FB08E623
:20140000FA08E6F922E6FF08E6FE08E6FD08E6FC22E6FB08E6FA08E6F908E6F822C5827092
:2014200002158314C58222740193F5F0E493F58385F08222E473EFF0A3EEF0A3EDF022EF58
:20144000F0A3EEF0A3EDF0A3ECF022EBF0A3EAF0A3E9F0A3E8F022E0FFA3E0FEA3E0FD2287
:20146000E0FFA3E0FEA3E0FDA3E0FC22E0FBA3E0FAA3E0F9A3E0F822E0FFA3E0FEC083A334
:20148000E004F0FD1582D08370030EEEF022E0FFA3E0FEC083A3E014F0FD1582D08304708B
:2014A000031EEEF0220D09292D000000008E6F00280A4170706C79206672657175656E63F1
:2014C00079203431304D487A204E4F5720616E642068697420616E79206B657920212121AF
:2014E000000A4672657175656E637920696E636F7272656374000A4D6F746F722061742017
:2015000073746F70706F696E74000A56616C7565203D2025752C2073746570203D2025759E
:20152000000A0A343130204D487A20506F736974696F6E203D20256909412F442076616C33
:201540007565203D202569000A41637475616C2073746570206E756D626572203D202569B2
:20156000000A4170706C79206672657175656E6379203432304D487A204E4F5720616E643D
:201580002068697420616E79206B657920212121000A0A343230204D487A20506F7369748A
:2015A000696F6E203D20256909412F442076616C7565203D202569000A4170706C7920663F
:2015C00072657175656E6379203433304D487A204E4F5720616E642068697420616E792085
:2015E0006B657920212121000A0A343330204D487A20506F736974696F6E203D20256909BC
:20160000412F442076616C7565203D202569000A0A343130204D487A20506F736974696FEF
:201620006E203D202569000A0A343230204D487A20506F736974696F6E203D202569000ACE
:201640000A343330204D487A20506F736974696F6E203D202569000A436F6D62696E657201
:2016600020636F6E7374616E742075707065722062616E64203D20256C69000A436F6D62DD
:20168000696E657220636F6E7374616E74206C6F7765722062616E64203D20256C69000A93
:2016A00043616C6962726174696F6E2073756363657366756C6C20212121000A43616C6963
:2016C00062726174696F6E206661696C6564202121212121000A466F7277617264203D2075
:2016E0002575205265666C656374203D20257520466F7277617264203D2025752C20566145
:201700006C7565203D20257520000A54756E696E672063617669747920256420746F20252C
:201720006C6920000A496E7075742074756E65206672657175656E63793A20000A496C6C47
:201740006567616C206672657175656E637920212121000A54756E696E67206361766974C5
:201760007920256420746F20256C69000A4D6F746F722068617320656E636F756E746572C0
:20178000656420612073746F70706F696E7400496C6C6567616C206672657175656E637943
:2017A000202121005E5A00082008005E430A0009090909090909536F667477617265207614
:2017C000657273696F6E3A2025730A00090909090909094861726477617265207665727330
:2017E000696F6E3A2025730A00094175746F6D6174696320544554524120436F6D62696EDF
:2018000065720909094D6F6465203A2025630A000909090909090954756E696E673A202512
:20182000630A0020204D61696E204D656E75097C0909537461747573206F662063617669EE
:20184000746965730A00313A2054756E6520636176697479097C20436176202020496E73A9
:20186000742E0954756E6564094672657109416C61726D0A00323A205061726B20636176B2
:20188000697479097C203109256309256309256C690925730A00333A2054756E65206E6F26
:2018A000205246097C203209256309256309256C690925730A00343A20787878782078784B
:2018C00078787878097C203309256309256309256C690925730A00353A2078787878207879
:2018E0007878787878097C203409256309256309256C690925730A00363A2054756E65209B
:201900007461626C65097C203509256309256309256C690925730A00373A2054696D6520D5
:201920006F7574097C203609256309256309256C690925730A00383A204D6F646509097CFF
:20194000203709256309256309256C690925730A00393A205574696C697479204D656E7524
:20196000097C203809256309256309256C690925730A00456E746572204D656E753A2000AD
:2019800020205574696C697479204D656E75097C0909537461747573206F6620636176698B
:2019A000746965730A00313A20446F776E6C6F6164097C20436176202020496E73742E09B1
:2019C00054756E6564094672657109416C61726D0A00323A204D6F7665206D6F746F7209F3
:2019E0007C203109256309256309256C690925730A00333A204D61737465722F736C61766C
:201A000065097C203209256309256309256C690925730A00343A20486172647761726520DE
:201A20007665722E7C203309256309256309256C690925730A00353A204465746563746F35
:201A400072097C203409256309256309256C690925730A00363A2044697361626C65207493
:201A6000756E2E097C203509256309256309256C690925730A00373A20787878782078782A
:201A800078787878097C203609256309256309256C690925730A00383A2043616C696272DC
:201AA000617465097C203709256309256309256C690925730A00393A204D61696E204D6556
:201AC0006E75097C203809256309256309256C690925730A00446576656C6F70204D656E67
:201AE000752021210A000A0909094D61696E204D656E752048656C700A00202046756E6327
:201B000074696F6E097C204465736372697074696F6E0A00313A2054756E652063617669EE
:201B20007479097C2054756E65732061206361766974792E20436176697479206E756D6243
:201B4000657220616E64206672657175656E6379206D75737420626520656E746572656492
:201B60002E0A0009097C2052465F706F77657220617420696E707574206578706563746508
:201B8000640A0009097C2053796E7461783A2078787878787820286B487A292E2049652EB0
:201BA00020343230313235203D203432302E313235204D487A0A0009097C20417661696C2A
:201BC00061626C6520696E206C6F63616C206D6F6465206F6E6C792E0A00323A20506172C1
:201BE0006B20636176697479097C205061726B732061206361766974792E204361766974AE
:201C000079206E756D626572206D75737420626520656E74657265640A0009097C2041765C
:201C200061696C61626C6520696E206C6F63616C206D6F646520616E64206175746F6D61F9
:201C4000746963206D6F64652E0A00333A2054756E65206E6F205246097C2054756E6573B5
:201C60002061206361766974792E20436176697479206E756D62657220616E64206672651C
:201C80007175656E6379206D75737420626520656E74657265642E0A00343A207878787832
:201CA000207878787878097C20526573657276656420666F72206C61746572207573652E8D
:201CC0000A00353A2078787878207878787878097C20526573657276656420666F72206C3B
:201CE00061746572207573652E0A00363A2054756E65207461626C65097C20446973706C9E
:201D0000617973206C61746573742074756E65207461626C657320666F7220616C6C20630F
:201D20006176697469657320696E7374616C6C65642E0A00373A2054696D65206F757409F5
:201D40007C205365742074696D65206F7574206265666F72652072657475726E696E6720C3
:201D6000746F206175746F6D61746963206D6F64652E2044656661756C742069730A0009B2
:201D8000097C203330206D696E2E0A0009097C2053796E7461783A2078787820286D696E1C
:201DA000292E203130203C3D20787878203C3D203132300A00383A204D6F646509097C200F
:201DC0005377697463686573206265747765656E206C6F63616C206D6F646520616E64204C
:201DE0006175746F6D61746963206D6F64652E0A0009097C204175746F6D61746963206D3D
:201E00006F646520697320726573756D65642061667465722054696D65206F75742E0A00E8
:201E2000393A205574696C697479204D656E75097C20476F657320746F20746865205574E6
:201E4000696C697479204D656E750A000A0909095574696C697479204D656E752048656C91
:201E6000700A00313A20446F776E6C6F6164097C20446F776E6C6F6164206E657720736FDC
:201E80006674776172652E20466F6C6C6F7720696E737472756374696F6E732E0A00323AFF
:201EA000204D6F7665206D6F746F72097C204D6F7665732061206D6F746F72206120676928
:201EC00076656E206E756D626572206F662073746570732E0A0009097C2043617669747976
:201EE000206E756D6265722C20646972656374696F6E20616E64206E756D626572206F663B
:201F0000207374657073206D75737420626520656E74657265642E0A00333A204D61737441
:201F200065722F736C617665097C20526573657276656420666F72206C61746572207573F4
:201F4000652E0A00343A204861726477617265207665722E7C204368616E6765732074683C
:201F6000652068617264776172652076657273696F6E206F662074686520636F6D62696E7A
:201F800065722E0A00353A204465746563746F72097C2050726F6772616D732074686520F8
:201FA0006465746563746F722E2043617669747920616E64206672657175656E6379206D37
:201FC0007573742062650A0009097C20656E74657265642E2053796E74617820666F7220C3
:201FE0006672657175656E63792078787878787820286B487A290A00363A20446973616204
:202000006C652074756E2E097C2044697361626C6573206175746F6D617469632074756E20
:20202000696E672E204175746F6D617469632074756E696E6720697320726573756D6564A7
:202040002061667465720A0009097C2054696D65206F75740A00373A207878787820787804
:20206000787878097C20526573657276656420666F72206C61746572207573652E0A003897
:202080003A2043616C696272617465097C20466163746F72792070726F6365647572652ECB
:2020A0002050726F7465637465642062792070617373776F72640A00393A204D61696E2086
:2020C0004D656E75097C20476F657320746F20746865204D61696E204D656E750A000A590D
:2020E0006F7520686176652063686F6F73656E20746F2074756E6520612063617669747919
:202100002066726F6D204D4D49000A546869732064697361626C6573206175746F6D6174C4
:2021200069632074756E696E67000A43686F6F736520436176697479206E756D626572205A
:20214000283129204361766974792031206F722028322920436176697479203220000A4923
:202160006E7075742074756E65206672657175656E63793A20000A496C6C6567616C206626
:2021800072657175656E637920212121000A4E6F20696E70757420706F77657220000A4979
:2021A0006C6C6567616C206672657175656E637920000A43616E206E6F742074756E652013
:2021C0006361766974792025632C2064756520746F205061726B696E67206661696C7572AB
:2021E0006520000A546869732066756E6374696F6E20697320617661696C61626C652069EC
:202200006E206C6F63616C206D6F6465000A43686F6F73652077686963682063617669748B
:202220007920746F207061726B3A2028412920416C6C2C2028312920436176697479203180
:20224000206F722028322920436176697479203220000A596F7520686176652063686F6F04
:2022600073656E20746F2074756E6520612063617669747920776974686F757420524620FC
:20228000706F776572000A43686F6F73652077686963682063617669747920746F207475B7
:2022A0006E6520283129204361766974792031206F72202832292043617669747920322022
:2022C000000A546869732066756E6374696F6E20697320617661696C61626C6520696E2002
:2022E0006C6F63616C206D6F6465206F6E6C79000A54756E65207461626C6520636176699B
:20230000747920313A200A00257520002A20000A54756E65207461626C6520636176697412
:202320007920323A200A000A4368616E67652073657474696E677320666F722074696D6557
:202340006F75742C2063757272656E746C79202575206D696E75746573000A496E707574F8
:20236000206E756D626572206F66206D696E757465733A20000A4E65772074696D656F7559
:20238000742073657474696E67203D20256C69206D696E75746573000A696C6C6567616C2B
:2023A00020696E70757420212121000A43686F6F73652073797374656D206D6F646520280D
:2023C0004C29204C6F63616C206F7220284129204175746F6D6174696320000A526566704C
:2023E0006F732020202020202020206361766974792031203D20256C69000A436D62436FB5
:202400006E7374207570706572206361766974792031203D20256C69000A436D62436F6E67
:202420007374206C6F776572206361766974792031203D20256C69000A526566706F73205B
:2024400020202020202020206361766974792032203D20256C69000A436D62436F6E737400
:20246000207570706572206361766974792032203D20256C69000A436D62436F6E73742054
:202480006C6F776572206361766974792032203D20256C69000A456E61626C6520646F77DF
:2024A0006E6C6F6164696E67206F66206E65772045435320736F6674776172652028592921
:2024C0002059657320284E29204E6F000A52657374617274696E6720626F6F742070726F9D
:2024E0006772616D000A43686F6F73652077686963682063617669747920746F206D6F7672
:202500006520283129204361766974792031206F722028322920436176697479203220002D
:202520000A43686F6F7365206D6F746F7220646972656374696F6E20285529205570206FC4
:20254000722028442920446F776E20000A496E707574206E756D626572206F662073746558
:2025600070733A20000A4D6F746F72206D6F76656420737563636566756C6C792021210007
:202580000A4D6F746F722068617320656E636F756E746572656420612073746F70706F6959
:2025A0006E74202121000A4D61737465722F536C6176652066756E6374696F6E206E6F7440
:2025C00020696D706C656D656E74656420000A496E707574206E65772048617264776172BA
:2025E00065207265766973696F6E206E756D62657220652E67205232412000253373000A4A
:20260000496E707574206465746563746F72206672657175656E63793A20000A5072657340
:20262000732028512920746F2071756974206D6573757265696E67000A44697361626C65D2
:202640002074756E696E67202844292064697361626C65206F722028452920656E61626C43
:202660006520000A496E7075742050617373776F72643A2000253473000A43616C696272CB
:202680006174696F6E206D6F6465000A43686F6F73652043617669747920746F2063616C0C
:2026A00069627261746520283129204361766974792031206F722028322920436176697465
:2026C00079203220000A50617373776F726420696E636F727265637420212121000A50618B
:2026E000726B696E672063617669747920256420001B5B324A001B5B4800253673000A4975
:202700006C6C6567616C2073796E7461782C2074727920616761696E200030313233343567
:202720003637383941424344454600286E756C6C20706F696E7465722900303132333435CA
:2027400036373839616263646566003F3F3F00C2D8C2D9C2DAC2DBC2DDC2E32275DA0078EE
:202760002CE4F608F630DC0280FBE5DAC403035403782EF6E5D975F004A4ADF01818CDF6F5
:20278000CD08F6FC08E6FEEC2EFCED34001818F608CCF6CCFD227872ECF67C0112681D7C18
:2027A0000212681DC2C87DB17E147F02128E7D1270C1786876017872E6146004E6B4031108
:2027C00090F912E0540F4410F0FC7D05126EB9800F90F912E0540F4420F0FC7D05126EB9A8
:2027E000786976007872E6FC12482D786A1213CB7872E6FC12482D786906786E1213CB78D5
:202800006A121411740512047270077869E624F650D2786DE62464FC18E63470FD30E70691
:20282000C3E49CFCE49DD3FDEC9403ED64809480400D7DE17E147F02128E7D7868760078F7
:2028400068E61460030230E390F912E0540F4440F0FC7D05126EB9126E2E783D7601786AD9
:20286000121405126C25783F76017872E6FE7F007D0E7CD81264BB7867ECF67872E61470EA
:202880000F90F911E04402F0FC7D06126EB98011E6B4020D90F911E04408F0FC7D06126ED2
:2028A000B97863E4F608F678677601785BF608F608760E0876D87865760E0876D87872E626
:2028C000FC7D0012312B785BEDF608ECF67864D396ED18964011EDF608ECF608E6FD08E69A
:2028E000785DCDF6CD08F6783F76017872E6FE7F01E4FD04FC1264BB7866E616187001166E
:202900000808ECF6700B7DF67E147F02128E7D80211818E6FD08E67942F7ED19F7785BE69D
:20292000FD08E67940F7ED19F77D0A7E157F02128E7D7867E660187864E624CEFC18E63428
:20294000FF785CFDECC396ED189650030228BD785EE616187001167872E614700F90F9111F
:20296000E054FDF0FC7D06126EB98011E6B4020D90F911E054F7F0FC7D06126EB97867E612
:202980001470367863E6FD08E67942F7ED19F7785DE6FD08E67940F7ED19F77D217E157F1F
:2029A00002128E7D7865E6FD08E67940F7ED19F77D487E157F02128E7D7868E61460030268
:2029C0002BE418E6146003022BE47D617E157F02128E7DC2C81270C17872E6146004E6B4A4
:2029E000031190F912E0540F4410F0FC7D05126EB9800F90F912E0540F4420F0FC7D051299
:202A00006EB9786976007872E6FC12482D786A1213CB7872E6FC12482D786906786E1213CE
:202A2000CB786A121411740512047270077869E624F650D2786DE624E8FC18E63479FD308C
:202A4000E706C3E49CFCE49DD3FDEC9403ED64809480400D7DE17E147F02128E7D78687660
:202A6000007868E6146003022BE490F912E0540F4440F0FC7D05126EB9126E2E783D760125
:202A8000786A121405126C25783F76017872E6FE7F017D037CE81264BB7867ECF618E62412
:202AA00018F618E634FCF67872E614700F90F911E04402F0FC7D06126EB98011E6B4020DDF
:202AC00090F911E04408F0FC7D06126EB97865E6FD08E67860F6ED18F67863E4F608F678E6
:202AE000677601785BF608F67872E6FC7D0012312B785BEDF608ECF67864D396ED189640BA
:202B000011EDF608ECF608E6FD08E6785FCDF6CD08F6783F76007872E6FE7F01E4FD04FC3D
:202B20001264BB7866E616187001160808ECF6700B7DF67E147F02128E7D80211818E6FD27
:202B400008E67942F7ED19F7785BE6FD08E67940F7ED19F77D0A7E157F02128E7D7867E60A
:202B600060187864E624CEFC18E634FF785CFDECC396ED18965003022AE87860E616187088
:202B800001167872E614700F90F911E054FDF0FC7D06126EB98011E6B4020D90F911E05440
:202BA000F7F0FC7D06126EB97867E61470367863E6FD08E67942F7ED19F7785FE6FD08E6F4
:202BC0007940F7ED19F77D917E157F02128E7D7865E6FD08E67940F7ED19F77D487E157FD7
:202BE00002128E7D7868E6146003022E0F18E6146003022E0F7DB87E157F02128E7DC2C896
:202C00001270C17872E6146004E6B4031190F912E0540F4410F0FC7D05126EB9800F90F98A
:202C200012E0540F4420F0FC7D05126EB9786976007872E6FC12482D786A1213CB7872E6E8
:202C4000FC12482D786906786E1213CB786A121411740512047270077869E624F650D27828
:202C60006DE624FAFC18E63482FD30E706C3E49CFCE49DD3FDEC9403ED64809480400D7D57
:202C8000E17E147F02128E7D786876007868E6146003022E0F90F912E0540F4440F0FC7D86
:202CA00005126EB9126E2E783D7601786A121405126C25783F76017872E6FE7F017D037CD4
:202CC000E81264BB7867ECF618E62418F618E634FCF67872E614700F90F911E04402F0FCB7
:202CE0007D06126EB98011E6B4020D90F911E04408F0FC7D06126EB97865E6FD08E67861E9
:202D0000CDF6CD08F608E4F608F678677601785BF608F67872E6FC7D0012312B785BEDF6BB
:202D200008ECF67864D396ED18964011EDF608ECF608E6FD08E67861CDF6CD08F6783F763E
:202D4000007872E6FE7F01E4FD04FC1264BB7866E616187001160808ECF6700B7DF67E1428
:202D60007F02128E7D80211818E6FD08E67942F7ED19F7785BE6FD08E67940F7ED19F77D96
:202D80000A7E157F02128E7D7867E660187864E624CEFC18E634FF785CFDECC396ED189629
:202DA0005003022D137862E616187001167872E614700F90F911E054FDF0FC7D06126EB933
:202DC0008011E6B4020D90F911E054F7F0FC7D06126EB97867E61470367863E6FD08E679A8
:202DE00042F7ED19F77861E6FD08E67940F7ED19F77DE87E157F02128E7D7865E6FD08E602
:202E00007940F7ED19F77D487E157F02128E7D7868E614600302304F18E614600302304F5B
:202E2000C37860795EE796FC1819E796FD120AF67A187B4B78807996120877120AB4787240
:202E4000E61425E025E02405F582E434FAF58312143FC378627960E796FC1819E796FD1233
:202E60000AF67A187B4B78807996120877120AB47872E61425E025E024FDF582E434F9F506
:202E80008312143F785DE6FD08E67940F7ED19F77D0F7E167F02128E7D785FE6FD08E67918
:202EA00040F7ED19F77D277E167F02128E7D7861E6FD08E67940F7ED19F77D3F7E167F02E0
:202EC000128E7D7872E61425E025E024FDF582E434F9F583121460EC783F1213CB7D577E5B
:202EE000167F02128E7D7872E61425E025E02405F582E434FAF583121460EC783F1213CBED
:202F00007D7B7E167F02128E7D7D9F7E167F02128E7D7872E6146003022FACE61425E025F1
:202F2000E024FDF582E434F9F583A3A3E0FFA3E0FE7C70124E857872E61425E025E0240502
:202F4000F582E434FAF583A3A3E0FFA3E0FE7C72124E857861E6FD08E6FCE4FEFF90F925C2
:202F600012143FE6FE18E6FF7C01124E857D597C00124DBC745990FA0FF0E490F90FF090EA
:202F8000F911E054FEF0FC7D06126EB9E490FA0EF090FA0EE0701290FA15E0700C78A6C608
:202FA0004401F6FC7D07126EB9023042E6B4020280030230421425E025E024FDF582E43446
:202FC000F9F583A3A3E0FFA3E0FE7C74124E857872E61425E025E02405F582E434FAF583ED
:202FE000A3A3E0FFA3E0FE7C76124E857861E6FD08E6FCE4FEFF90F92912143FE6FE18E6D4
:20300000FF7C0B124E857D597C0A124DBC745990FA16F0E490F910F090F911E054FBF0FC4F
:203020007D06126EB9E490FA15F090FA0EE0701290FA15E0700C78A6C64401F6FC7D0712BB
:203040006EB97872E6FC12681D1270C10230DA7DBB7E167F02128E7D7872E614700F90F941
:2030600011E04401F0FC7D06126EB98011E6B4020D90F911E04404F0FC7D06126EB978A6B0
:20308000C654FEF6FC7D07126EB97872E6FC12681D7872E614700F90F911E04401F0FC7D7B
:2030A00006126EB98011E6B4020D90F911E04404F0FC7D06126EB978A6C654FEF6FC7D0781
:2030C000126EB97872E61475F007A4240EF582E434FAF5837404F01270C17872E6FC126B9C
:2030E000F78047E670447DBB7E167F02128E7D7872E614700F90F911E04401F0FC7D06126B
:203100006EB98011E6B4020D90F911E04404F0FC7D06126EB978A6C654FEF6FC7D07126EB8
:20312000B9740490FA15F01270C122784AE4F608F608F608F608F608F67856760008760016
:203140000876000808EDF618ECF624FD4004C2F88002D2F8EC14701190F912E054F0440114
:20316000F0FC7D05126EB98013ECB4020F90F912E054F04404F0FC7D05126EB97857E660A1
:20318000030233AC18E660030233AC0808E624F650030233ACD294D290784AE4F608F6085B
:2031A000F608F608F608F608F608F67859E6146004E6B4032F7850E6FF08E6FE209410C308
:2031C000EE9494EF941150070EBE00010F80ED7850EFF608EEF6C39493EF9411400478567C
:2031E0007601802D7850E6FF08E6FE209010C3EE9494EF941150070EBE00010F80ED78507D
:20320000EFF608EEF6C39493EF9411400478567601D37851E6940A18E69400401AE4FEFFE9
:20322000C3EE9464EF940050070EBE00010F80F07854EFF608EEF67856E660030233A61818
:2032400018E4F608F6C37855E6941418E69400501612275C784BE62CF618E63DF678550604
:20326000E61870010680DE7859E614701190F912E054F04402F0FC7D05126EB98013E6B456
:20328000020F90F912E054F04408F0FC7D05126EB9E4FEFFC3EE9464EF940050070EBE003B
:2032A000010F80F07854EFF608EEF6E4FF18F608F6C37855E6941418E69400501612275C57
:2032C000784DE62CF618E63DF6785506E61870010680DE7859E614701190F912E054F044FB
:2032E00001F0FC7D05126EB98013E6B4020F90F912E054F04404F0FC7D05126EB9E4FEFF59
:20330000C3EE9464EF940050070EBE00010F80F07854EFF608EEF6E4FF18F608F6C37855C2
:20332000E6941418E69400501612275C784FE62CF618E63DF6785506E61870010680DE7854
:2033400059E6146004E6B4032B309428C3784F794BE796FC1819E796FD30E706C3E49CFC34
:20336000E49DC3FDEC9420ED648094835004785776018032E664026004E6B40429309026DB
:20338000C3784F794BE796FC1819E796FD30E706C3E49CFCE49DC3FDEC9420ED6480948396
:2033A00050047857760178580602317CE4FB7A14784AE6F908E6F81201FDE4FB7A14E8781D
:2033C0004BF6E918F6784CE6F908E6F81201FDE4FB7A14E8784DF6E918F6784EE6F908E682
:2033E000F81201FDE8784FF6E918F6784BE624F4FC18E63401C3FD784DEC96FC18ED967823
:2034000052F608ECF6785AE61470397852E6FD08E67946F7ED19F7784EE6FD08E67944F76C
:20342000ED19F7784CE6FD08E67942F7ED19F7784AE6FD08E67940F7ED19F77DD57E167FA6
:2034400002128E7D7857E61470087852E6FD08E6FC22E4FCFD2278607601786376007866D6
:2034600076007869E4F608F67879F608F608F608F608F608F608F608F67889ECF6147008D5
:2034800090F90FE024FE5014ECB402028003023F6D90F910E024FE5003023F6DEC14703A13
:2034A00090FA0DE0B4503390F9FD12146090F92512146C1202EE7B19794778807AA1120592
:2034C00020120B0C7A187B56785A7996120877120AB490F91D12143F803CECB4023890FAD3
:2034E00014E0B4503190FA0112146090F92912146C1202EE7B19794778807AA1120520129C
:203500000B0C7A187B56785A7996120877120AB490F92112143F786176007889E6FC124854
:203520002D786D1213CB7889E6FC12482D78610678711213CB786D121411740512047270DA
:20354000077861E624F650D2786D121405E4FB04FA04F8797D041204726003023F6B798FE7
:20356000789F740F1204726003023F6B7861E624F65003023F6B7889E6147037ECFAEDFBD2
:20358000C390F924E09AF890F923E09BF930E706C3E498F8E499D3F9E8941DE96480948012
:2035A000401190F91D12146078751213CB78637601803B7889E6B40235ECFAEDFBC390F9B8
:2035C00020E09AF890F91FE09BF930E706C3E498F8E499D3F9E8941DE964809480400F9047
:2035E000F92112146078751213CB78637601C378787970E796FC1819E796FD30E706C3E478
:203600009CFCE49DD3FDEC9404ED648094804004786676017866E61470067863E614601A22
:203620007889E61475F007A4240DF582E434FAF583E0B474028003023F6B90F912E0540F36
:203640004440F0FC7D05126EB9126E2E783D7601786D121405126C257889E61475F007A4A7
:20366000240DF582E434FAF583E0647460067863E61460127866E6146003023A237863E658
:20368000146003023A23786D121405120B0C7A187B56785A79961208777A7A7B4412086F0A
:2036A000120AB478711213CB78411213CB7889E6783F760008F67D0A7E177F02128E7D7478
:2036C0000190F919F0786D121405E4FB04FA78187986740F12047270707875121405781848
:2036E000740F12047270627889E61425E025E024FDF582E434F9F583121460120B0C7A1886
:203700007B56785A7996120877786D121411120B63C8C0E078851213CBD0E0C812088378E8
:2037200075121411120B6312136212138378851214051213A71208831213A712099E120AFC
:20374000B478811213CB023994786D1214057818740312047270707875121405781874035F
:2037600012047270627889E61425E025E02405F582E434FAF583121460120B0C7A187B56AE
:20378000785A7996120877786D121411120B63C8C0E078851213CBD0E0C8120883787512B2
:2037A0001411120B6312136212138378851214051213A71208831213A712099E120AB478D7
:2037C000811213CB023994786D1214057818740B12047260030238AF78751214057818749A
:2037E0000712047260030238AF7889E61425E025E02405F582E434FAF583121460120B0C10
:203800007A187B56785A79961208777875121411120B63C8C0E078851213CBD0E0C8120848
:20382000831213627885121405E4F8790C7B477AC31208831213A71209AA120AB47889E611
:203840001425E025E024FDF582E434F9F58312146C120B63C8C0E078811213CBD0E0C87ED0
:20386000187F567C5A7D96120883786D121411120B63C8C0E078851213CBD0E0C8120883CF
:203880001213627885121405E4F8790C7B477AC31208831213A712099E7881121411120BAA
:2038A0004E1209B7120AB478811213CB023994786D1214057818740712047260030239948B
:2038C00078751214057818740B12047260030239947889E61425E025E024FDF582E434F959
:2038E000F583121460120B0C7A187B56785A79961208777875121411120B63C8C0E07885C3
:203900001213CBD0E0C81208831213627885121405E4F8790C7B477AC31208831213A71218
:2039200009AA120AB47889E61425E025E02405F582E434FAF58312146C120B63C8C0E078E3
:20394000811213CBD0E0C87E187F567C5A7D96120883786D121411120B63C8C0E07885127A
:2039600013CBD0E0C81208831213627885121405E4F8790C7B477AC31208831213A71209C1
:203980009E7881121411120B4E1209B7120AB478811213CB7889E614700F90F911E0440229
:2039A000F0FC7D06126EB98011E6B4020D90F911E04408F0FC7D06126EB97883E6FD08E6EB
:2039C000786BCDF6CD08F6C39419ED64809480401C783F7600786CE624E7FC18E634FFFD99
:2039E0007889E6FE7F011264BB7860ECF6C3786CE6941918E6648094805028783F7601E4BD
:203A0000FD7419C3786C96FC18ED96FD30E706C3E49CFCE49DFD7889E6FE7F001264BB7864
:203A200060ECF67860E6146003023CA87889E6FC124612740190F919F07860ECF6146003A4
:203A4000023BD07889E6FC1247C57861ECF67889E6FC12475C7889E61475F064A4FD7861C7
:203A6000E625E02D242DF582E434F9F583E0FFA3E0FE7889E61475F064A47862CCF6CCFDB0
:203A8000EC25E02D242DF582E434F9F583C3A3E0FCEE9C786AF612141DE0FCEF9C18F6C398
:203AA00008E6941E18E694005003023BCD7861E624F65008E624D84003023BCDE624F640D7
:203AC00017783F76017889E6FE7F00E4FD7C4B1264BB7860ECF68015783F76017889E6FE02
:203AE0007F00E4FD7C191264BB7860ECF67889E6FC124612740190F919F07860ECF6147054
:203B00005E7889E6FC1247C57861ECF67889E6FC12475C7889E61475F064A4FD7861E625AA
:203B2000E02D242DF582E434F9F583E0FFA3E0FE7889E61475F064A47862CCF6CCFDEC25E9
:203B4000E02D242DF582E434F9F583C3A3E0FCEE9C786AF612141DE0FCEF9C18F6806EECD1
:203B600064026004ECB40365ECB40211783F76007889E6FE7F01E4FD7C191264BB7889E6A0
:203B8000147024786D12140590F91D12143FE6FE18E6FF7C04124E857D747C03124DBC741D
:203BA0007490FA0DF08026E6B40222786D12140590F92112143FE6FE18E6FF7C0E124E8537
:203BC0007D747C0D124DBC747490FA14F0023CA8EC64026009ECB403028003023CA878892A
:203BE000E61475F007A4240DF582E434FAF583E0B4740A7866E67005E490F919F0ECB40226
:203C000011783F76007889E6FE7F01E4FD7C191264BB7889E6147047786D12140590F91DF2
:203C200012143FE6FE18E6FF7C04124E85786D121405120B0C7A187B56785A7996120877CB
:203C40007A7A7B4412086F120AB490FA1012143F7D747C03124DBC747490FA0DF08049E6B0
:203C6000B40245786D12140590F92112143FE6FE18E6FF7C0E124E85786D121405120B0CA1
:203C80007A187B56785A79961208777A7A7B4412086F120AB490FA1712143F7D747C0D12B1
:203CA0004DBC747490FA14F0C3786AE6942818E694005003023EDE7860E6146003023EDEE8
:203CC0007889E61475F064A4FC7861E625E02C242DF582E434F9F583A3E024F97868F612B7
:203CE000141DE034FF18F67861E61818F6FF1F7889E61475F064A4FCEF25E02C242DF58223
:203D0000E434F9F583C37868A3E096FC1812141DE096D3FDEC9407ED940040D2785FEFF6EB
:203D20007864F67861E6FF0F7889E61475F064A4FCEF25E02C242DF582E434F9F583C378D4
:203D400068A3E096FC1812141DE096D3FDEC9407ED940040D2785FEFF6FC786426FEE4335C
:203D6000FFE4FB7A02120182E87868F6E918F67865ECF61826FCE433FDE4FB7A021201C460
:203D8000E84960497889E61475F064A4FC7865E625E02C242DF582E434F9F583E0FDA3E040
:203DA000FC7889E61475F064A4FE7864E625E02E242DF582E434F9F583E0FFA3E0FEECC34C
:203DC0009EED9F4008786806E6187001067889E61470177865E61826FCE433FDE4FB7A0228
:203DE000120189E890F91BF08019E6B402157865E61826FCE433FDE4FB7A02120189E890E1
:203E0000F91CF0783F7601E4FD7431C3786896FC18ED96FD7889E6FE7F001264BB7860ECC3
:203E2000F67889E6147059786D12140590F91D12143FE6FE18E6FF7C04124E85786D12145C
:203E400005120B0C7A187B56785A79961208777A7A7B4412086F120AB490FA1012143F7DD7
:203E6000547C03124DBC745490FA0DF090F911E054FDF0FC7D06126EB9E490F90FF0805B4B
:203E8000E6B40257786D12140590F92112143FE6FE18E6FF7C0E124E85786D121405120B93
:203EA0000C7A187B56785A79961208777A7A7B4412086F120AB490FA1712143F7D547C0DB5
:203EC000124DBC745490FA14F090F911E054F7F0FC7D06126EB9E490F910F0023F6B7889EA
:203EE000E61475F007A4240DF582E434FAF583E0B47432C3786AE6942818E694005026E617
:203F0000084660217889E6FC12681D7889E614700890F90FE004F0800AE6B4020690F910B4
:203F2000E004F080467889E614700F90F90FE024FE400790FA0DE0B47414E6B4022D90F987
:203F400010E024FE402590FA14E06474601DE6FC12681D7889E614700890F90FE004F0803F
:203F60000AE6B4020690F910E004F0805278A6C654FEF6FC7D07126EB97889E614701C905A
:203F8000F911E04401F0FC7D06126EB97D017C06124DBC740190FA0EF0801EE6B4021A904E
:203FA000F911E04404F0FC7D06126EB97D017C10124DBC740190FA15F0740190F919F0787F
:203FC00089E6FC026BF77895ECF67D247E177F02128E7D126FD9787D1213CB788D7600E4B1
:203FE000FB7A06794178907403120472700B798F78B074071204727015EC4D4E4F600C7D93
:204000003C7E177F02128E7D1270C1024611787D121405E4FA790378E81202EE120B0C7A16
:20402000187B56785A7996120877120AB4787D1213CB7895E614705890FA0DE0B45051E6EF
:204040001425E025E024FDF582E434F9F58312146090F92512146C1202EE7B19794778800D
:204060007AA1120520120B0C7A187B56785A7996120877120AB490F91D12143F90FA14E097
:20408000B4500B90F921E4F0A3F0A3F0A3F0805AE6B4025690FA14E0B4504FE61425E02519
:2040A000E024FDF582E434F9F58312146090F92912146C1202EE7B19794778807AA11205B5
:2040C00020120B0C7A187B56785A7996120877120AB490F92112143F90FA0DE0B4500B90CD
:2040E000F91DE4F0A3F0A3F0A3F07895E6147036C3788090F924E096FC1890F923E096FD5F
:2041000030E706C3E49CFCE49DC3FDEC9421ED64809480401190F91D12146008081213CBFF
:20412000788D7601803A7895E6B40234C3788090F920E096FC1890F91FE096FD30E706C383
:20414000E49CFCE49DC3FDEC9421ED64809480400F90F92112146008081213CB788D760121
:20416000788DE61460030245FF787D121405120B0C7A187B56785A79961208777A7A7B44C6
:2041800012086F120AB478851213CB78411213CB7895E6783F760008F67D537E177F02121A
:2041A0008E7D787D121405E4FB04FA78187986740F120472707078811214057818740F1234
:2041C000047270627895E61425E025E024FDF582E434F9F583121460120B0C7A187B5678DB
:2041E0005A7996120877787D121411120B63C8C0E078891213CBD0E0C8120883788112148C
:2042000011120B6312136212138378891214051213A71208831213A712099E120AB4788FED
:204220001213CB024471787D12140578187403120472707078811214057818740312047295
:2042400070627895E61425E025E02405F582E434FAF583121460120B0C7A187B56785A79F4
:2042600096120877787D121411120B63C8C0E078891213CBD0E0C8120883788112141112BB
:204280000B6312136212138378891214051213A71208831213A712099E120AB4788F12136B
:2042A000CB024471787D1214057818740B120472600302438C788112140578187403120450
:2042C00072600302438C7895E61425E025E02405F582E434FAF583121460120B0C7A187B41
:2042E00056785A79961208777881121411120B63C8C0E078891213CBD0E0C81208831213B3
:20430000627889121405E4F8790C7B477AC31208831213A71209AA120AB47895E61425E0A5
:2043200025E024FDF582E434F9F58312146C120B63C8C0E0788F1213CBD0E0C87E187F5603
:204340007C5A7D96120883787D121411120B63C8C0E078891213CBD0E0C812088312136236
:204360007889121405E4F8790C7B477AC31208831213A712099E788F121411120B4E1209CB
:20438000B7120AB4788F1213CB024471787D12140578187407120472600302447178811210
:2043A00014057818740F12047260030244717895E61425E025E024FDF582E434F9F58312EB
:2043C0001460120B0C7A187B56785A79961208777881121411120B63C8C0E078891213CB62
:2043E000D0E0C81208831213627889121405E4F8790C7B477AC31208831213A71209AA1255
:204400000AB47895E61425E025E02405F582E434FAF58312146C120B63C8C0E0788F1213FD
:20442000CBD0E0C87E187F567C5A7D96120883787D121411120B63C8C0E078891213CBD073
:20444000E0C81208831213627889121405E4F8790C7B477AC31208831213A712099E788FDB
:20446000121411120B4E1209B7120AB4788F1213CB7895E614700F90F911E04402F0FC7D52
:2044800006126EB98011E6B4020D90F911E04408F0FC7D06126EB97891E6FD08E608CDF690
:2044A000CD08F6D39400ED648094804016783F76007893E608E6FC08E6FE7F011264BB7872
:2044C0008EECF67893E6335022783F76017893E6FD08E6FCED30E706C3E49CFCE49DFD0801
:2044E000E6FE7F001264BB788EECF67895E6FC126BF7788EE670127D6C7E177F02128E7D53
:204500007895E6FC12681D80147895E61475F007A4240DF582E434FAF583744DF07895E694
:2045200014706C90F911E054FDF0FC7D06126EB97D4D7C03124DBC787D12140590F91D12DC
:20454000143FE6FE18E6FF7C04124E85787D121405120B0C7A187B56785A79961208777A2A
:204560007A7B4412086F120AB490FA1012143F90FA0EE06018E490FA0EF07D007C06124DF0
:20458000BC78A6C64401F6FC7D07126EB9806EE6B4026A90F911E054F7F0FC7D06126EB926
:2045A0007D4D7C0D124DBC787D12140590F92112143FE6FE18E6FF7C0E124E85787D1214F3
:2045C00005120B0C7A187B56785A79961208777A7A7B4412086F120AB490FA1712143F9036
:2045E000FA15E06018E490FA15F07D007C06124DBC78A6C64401F6FC7D07126EB9800C7DE6
:204600008F7E177F02128E7D1270C1740190F919F022785C760108760108ECF61CEC75F04B
:2046200007A4240DF582E434FAF583E0B4742BE6FC7D0012312BD3EC9403ED9400401778F7
:204640003F7601785EE6FE7F00E4FD7C191264BB785CECF68004785D7600785CE61460030E
:2046600002475108E614600302475118187600785BE624CE4063783F7600785EE6FE7F0146
:20468000E4FD04FC1264BB785CECF67002804A0808E6FC7D0012312B785EE61475F064A4FC
:2046A000FE785BE625E02E242DF582E434F9F583EDF0A3ECF0785EE61475F064A4FC785B57
:2046C000E625E02C242DF582E434F9F583E0FDA3E04D70028003068096785BE6B4320214FF
:2046E000F608E670037C00220808E61475F064A4FC785BE625E02C242DF582E434F9F58317
:20470000E0FDA3E04D7047E624E74020E6601D783F76007D00FCE4FF7419C39CFCEF9DFD87
:20472000785EE6FE7F011264BB7C0322E624E6501A783F7601785BE624E7FCE434FFFD7899
:204740005EE6FE7F001264BB7C03227C02227C0122785DE670037C03227C0022782E7604FA
:2047600008E4F6782C76007830ECF6782CE6FFEF24CE4045EC1475F064A4FDEF25E02D2415
:204780002DF582E434F9F583E0FBA3E0782FC396EB18965021EC1475F064A4FDEF25E02DF9
:2047A000242DF582E434F9F583E0FBA3E0CBF6CB08F61818EFF60F80B67830ECF6782CEF49
:2047C000F608E6FC22782EE4F608F6782C76007830ECF6782CE6FFEF24CE4045EC1475F061
:2047E00064A4FDEF25E02D242DF582E434F9F583E0FBA3E0782FD396EB18964021EC147565
:20480000F064A4FDEF25E02D242DF582E434F9F583E0FBA3E0CBF6CB08F61818EFF60F80A5
:20482000B67830ECF6782CEFF608E6FC22C2C8E490F913F090F914F07841ECF6126DEEC252
:20484000F97839E4F608F608F608F608F608F608F608F67836760090F914E0600302499102
:2048600090F913E060030249917836E624F65003024991D2FDC2EAD2FCC2FAD2FBC2FB759C
:204880008A00758C00758B00758D00D28ED2B4E4F090F914F07839F608F608F608F67835F6
:2048A00076807841E624FD4004C2F88002D2F8D294D2907837E4F608F67841E6146004E6AC
:2048C000B4034090F912E0540F4410F0FC7D05126EB97837E6FF08E6FE209410C3EE9494EB
:2048E000EF941150070EBE00010F80ED7837EFF608EEF6C39493EF94114006740190F9132F
:20490000F0803E90F912E0540F4420F0FC7D05126EB97837E6FF08E6FE209010C3EE9494E7
:20492000EF941150070EBE00010F80ED7837EFF608EEF6C39493EF94114006740190F913EE
:20494000F090F913E0704430B40280FBD2FAD28CE58A24F0400280F8C2FAE58A24EF4002EF
:2049600080F8C28C7841E6146004E6B4030B309408740190F914F08012E664026004E6B408
:204980000409309006740190F914F078360602485790F914E0146003024A1CC28EC2FCD2B1
:2049A000FC30FD0D7835E6FCE4FDFEFF78391205717835C6C313F60808E4F608F6C3783881
:2049C000E6940718E694005026D2FDD2EAC2EA30FD0D1818E6FCE4FDFEFF7839120571783C
:2049E00035C6C313F6783806E61870010680CEAC8BE4FDFEFF783D1213CB783D7C0912056C
:204A0000A630B509E4FCFEFF04FD1205711214057839120571D2FBC2FBD2C822D2C8E4FC78
:204A2000FDFEFF22758955C28CC28EC2FAD2FBC2FBD2FCD2B4D2B5C2EA227C017D002290CE
:204A4000F9F9E0FDA3E07831CDF6CD08F6782C7680087600783076007832E6240AFC18E6DF
:204A60003400FD90F9FAE0D39C90F9F9E09D4005D2981876013098E07830E6703BC29818A3
:204A800018A69918E6FD18E6FF7E00EE24F8400FEF782E566F70010DEFC313FF0E80EC7862
:204AA0002DEDF60808EEF6782CEFF6ED20E006E599547FFC227C00227C0D22782C1213B93C
:204AC000782C1213F3121011601312134B782C1213B91210077D00FC126E9980E32290F9B9
:204AE0000BE024B8F582E434F8F583E0602290F90AE0FDA3E0FCE004F090F90A7003E004E1
:204B0000F0EC24B8F582E434F8F583E07D00FC2290F90AE4F0A3F0124A3F7833ECF6B41A73
:204B20001890F90AE0FDA3E04D700E7DA47E177F02124ABB74FFFCFD22E6B47F2190F90AF6
:204B4000E0FDA3E04D6014E024FFF090F90AE034FFF07DA77E177F02124ABB024BFAB4035C
:204B6000157DAB7E177F02124ABB90F90AE4F0A37451F0024BFDB40D3E90F90AE0FDA3E0D0
:204B8000FCE004F090F90A7003E004F0EC24B8F582E434F8F583740AF0E4FD7C0A126E99B6
:204BA00090F90BE024B8F582E434F8F583E4F090F90AF0A3F08046C390F90BE0945090F952
:204BC0000AE064809480502BE624E05024E6FEE0FDA3E0FCE004F090F90A7003E004F0EC40
:204BE00024B8F582E434F8F583EEF07D00FC126E998007E4FD7C07126E99024B17024ADED8
:204C000022D295D296782C760030950F30960C124C00C295124C00C29680027601782CE6F5
:204C2000FC22C295124C00D296124C00D29522782DECF654806480600274FF04A2E0920026
:204C4000187600782CE624F8401FA200929508C625E0F6D296E654806480600274FF04A2AE
:204C6000E09200C296180680DAD295024C00D295124C00782DE4F6087680087600782C7663
:204C80000008E6FD08E6FC1818E6FFEF24F84021D296EF6007EDC313FDEC13FCA29592007C
:204CA000C296300009EC782FFEE64E792FF70F80DA782DEDF608ECF61818EFF6782FE6FC86
:204CC00022C295124C00D296124C00C296124C00D295024C00D296124C00A2959200782C99
:204CE0007600E6FF300008EF24FB40030F80F5782CEFF6C296A20022D295124C00D2961268
:204D00004C00C296024C00E490F90EF07831760108ECF67831E614701A90F90EE024FB4029
:204D200012124C017831ECF614700690F90EE004F080E0E6702DE490F90EF07CA0124C2F8B
:204D4000124CD5920140167832E6FC124C2F124CD59201500690F90EE004F0800690F90E7A
:204D6000E004F090F90EE07045783176017831E6601A90F90EE024FB4012124C017831EC2E
:204D8000F614700690F90EE004F080E17CA1124C2F124CD59201500690F90EE004F090F90D
:204DA0000EE0700A124C6E7830ECF6124CF890F90EE07003124C227830E6FC22782E7600AD
:204DC0000876017833EDF618ECF6782FE6601418E624FB400E124C01782FECF614700218DA
:204DE0000680E7782FE670357CA0124C2F124CD5782E7600920140227832E6FC124C2F12FC
:204E00004CD59201400C7833E6FC124C2F124CD59201300103782E06800106800218061299
:204E20004C22E4FEFFC3EE94E8EF940350070EBE00010F80F07830EFF608EEF6782EE6FCCC
:204E4000227836ECF6124D077835ECF61818E4F608F690F90EE07029EC18F608E4F60808A7
:204E6000E604FC124D077835ECF690F90EE0700D18E64CF618E6F6E6FD08E6FC22E4FCFD63
:204E800022E4FCFD22E490F90EF07838EFF608EEF6EF7836F618760008E61818F67837CC55
:204EA000F6CCFD124DBCEC90F90EF0701D7839E6FC7835760008CCF6CC1818F6FD7837E614
:204EC00004FC124DBCEC90F90EF022E490F91AF090F918F0744190F915F0744590F916F08F
:204EE000E490F919F0C29390F911F078A676FF90F912F090F90FF090F910F07C01126BF73D
:204F00007C02126BF7E490F917F0C2EFC2E812709912274F124A24126F07126DEE90F9121D
:204F2000E054F0F0FC7D05126EB9E490F911F07D06FC126EB978A6C654FBF6FC7D07126E57
:204F4000B978A5760078A5E624FD4018E62468FC124D0778A5E624F5F582E434F9F583ECAD
:204F6000F00680E190F9F5E06458601B90F9F5E064526013742090F9F5F090F9F6F090F9C4
:204F8000F7F0E490F9F8F090F9FB7407F0A304F090F9F9E4F0A3F0D2C8D2ADD2991261D09F
:204FA000740190FA47F0C29890FA0DE0B44D0C90F916E0B445057C0112681D90FA14E0B41A
:204FC0004D0C90F916E0B445057C0212681D90FA0EE0701890FA0FE0B4591190F916E0B41C
:204FE000450A7C011234567C01126BF790F918E0147003126C1590F919E014700D90FA47D9
:20500000E0FC1250CAE490F919F090F916E0B4451AE4FEFFC3EE9450EF94C350070EBE00A1
:20502000010F80F078A3EFF608EEF690FA15E0701890FA16E0B4591190F916E0B4450A7C61
:20504000021234567C02126BF790F918E0147003126C1590F919E014700D90FA47E0FC1253
:2050600050CAE490F919F090F916E0B4451AE4FEFFC3EE9450EF94C350070EBE00010F809F
:20508000F078A3EFF608EEF690FA0DE0B4541A90FA14E0B4541390F915E0B4410C78A6C69F
:2050A0004402F6FC7D07126EB93098181270C1EC90F90CF012581090FA47E0FC1250CAE430
:2050C00090F919F0024FA880FE22784B908F57790F121311785AECF6126FC7784A76007802
:2050E0005AE6120D410104580F50F3537A5601560D5713783F760208768F08764E7DAF7EBE
:20510000177F02128E7D783F76010876F90876F57DCC7E177F02128E7D90F915E0783F769B
:205120000008F67DE97E177F02128E7D90F916E0783F760008F67D107E187F02128E7D78F5
:205140004A7600784AE624B0400CE4FD7C2D126E99784A0680ED7D237E187F02128E7D78A3
:205160004A7600784AE624B0400CE4FD7C2D126E99784A0680ED7D467E187F02128E7D9048
:20518000FA0EE075F003A4244BFDE4FEFF78471213B990FA1012146078431213CB90FA0DCF
:2051A000E07841760008F690FA0FE0783F760008F67D757E187F02128E7D90FA15E075F034
:2051C00003A4244BFDE4FEFF78471213B990FA1712146078431213CB90FA14E078417600BF
:2051E00008F690FA16E0783F760008F67D967E187F02128E7D90FA1CE075F003A4244BFDC1
:20520000E4FEFF78471213B990FA1E12146078431213CB90FA1BE07841760008F690FA1DDE
:20522000E0783F760008F67DB67E187F02128E7D90FA23E075F003A4244BFDE4FEFF784757
:205240001213B990FA2512146078431213CB90FA22E07841760008F690FA24E0783F76001C
:2052600008F67DD77E187F02128E7D90FA2AE075F003A4244BFDE4FEFF78471213B990FA94
:205280002C12146078431213CB90FA29E07841760008F690FA2BE0783F760008F67DF87E3E
:2052A000187F02128E7D90FA31E075F003A4244BFDE4FEFF78471213B990FA3312146078EC
:2052C000431213CB90FA30E07841760008F690FA32E0783F760008F67D187E197F02128EC0
:2052E0007D90FA38E075F003A4244BFDE4FEFF78471213B990FA3A12146078431213CB9014
:20530000FA37E07841760008F690FA39E0783F760008F67D367E197F02128E7D90FA3FE0F0
:2053200075F003A4244BFDE4FEFF78471213B990FA4112146078431213CB90FA3EE078411A
:20534000760008F690FA40E0783F760008F67D517E197F02128E7D784A7600784AE624B04D
:20536000400CE4FD7C2D126E99784A0680ED7D737E197F02128E7D02580F783F76020876CE
:205380008F08764E7DAF7E177F02128E7D783F76010876F90876F57DCC7E177F02128E7DBF
:2053A00090F915E0783F760008F67DE97E177F02128E7D90F916E0783F760008F67D107EF6
:2053C000187F02128E7D784A7600784AE624B0400CE4FD7C2D126E99784A0680ED7D807EC4
:2053E000197F02128E7D784A7600784AE624B0400CE4FD7C2D126E99784A0680ED7DA67E7D
:20540000197F02128E7D90FA0EE075F003A4244BFDE4FEFF78471213B990FA1012146078CF
:20542000431213CB90FA0DE07841760008F690FA0FE0783F760008F67DD27E197F02128EEA
:205440007D90FA15E075F003A4244BFDE4FEFF78471213B990FA1712146078431213CB90F8
:20546000FA14E07841760008F690FA16E0783F760008F67DF27E197F02128E7D90FA1CE03C
:2054800075F003A4244BFDE4FEFF78471213B990FA1E12146078431213CB90FA1BE07841FF
:2054A000760008F690FA1DE0783F760008F67D147E1A7F02128E7D90FA23E075F003A42442
:2054C0004BFDE4FEFF78471213B990FA2512146078431213CB90FA22E07841760008F690DD
:2054E000FA24E0783F760008F67D367E1A7F02128E7D90FA2AE075F003A4244BFDE4FEFFAD
:2055000078471213B990FA2C12146078431213CB90FA29E07841760008F690FA2BE0783FFB
:20552000760008F67D547E1A7F02128E7D90FA31E075F003A4244BFDE4FEFF78471213B95F
:2055400090FA3312146078431213CB90FA30E07841760008F690FA32E0783F760008F67D52
:20556000767E1A7F02128E7D90FA38E075F003A4244BFDE4FEFF78471213B990FA3A1214FD
:205580006078431213CB90FA37E07841760008F690FA39E0783F760008F67D977E1A7F0237
:2055A000128E7D90FA3FE075F003A4244BFDE4FEFF78471213B990FA4112146078431213FE
:2055C000CB90FA3EE07841760008F690FA40E0783F760008F67DB67E1A7F02128E7D784A2B
:2055E0007600784AE624B0400CE4FD7C2D126E99784A0680ED7D737E197F02128E7D025816
:205600000F7DD57E1A7F02128E7D02580F7DE67E1A7F02128E7D784A7600784AE624B040FD
:205620000CE4FD7C2D126E99784A0680ED7DFA7E1A7F02128E7D784A7600784AE624B040E5
:205640000CE4FD7C2D126E99784A0680ED7D147E1B7F02128E7D7D637E1B7F02128E7D7D0A
:20566000837E1B7F02128E7D7DB77E1B7F02128E7D7DDA7E1B7F02128E7D7D1A7E1C7F02C5
:20568000128E7D7D4B7E1C7F02128E7D7D997E1C7F02128E7D7DC27E1C7F02128E7D7DEBC0
:2056A0007E1C7F02128E7D7D1A7E1C7F02128E7D7D347E1D7F02128E7D7D7F7E1D7F0212CF
:2056C0008E7D7D8C7E1D7F02128E7D7DB77E1B7F02128E7D7DB57E1D7F02128E7D7DF17EBB
:2056E0001D7F02128E7D7D207E1E7F02128E7D784A7600784AE624B0400CE4FD7C2D126E0E
:2057000099784A0680EDC2981270C1EC90F90CF002580F7D4C7E1E7F02128E7D784A760009
:20572000784AE624B0400CE4FD7C2D126E99784A0680ED7DFA7E1A7F02128E7D784A7600E4
:20574000784AE624B0400CE4FD7C2D126E99784A0680ED7D637E1E7F02128E7D7DB77E1BC2
:205760007F02128E7D7D9E7E1E7F02128E7D7DD67E1E7F02128E7D7D1A7E1C7F02128E7DDA
:205780007D197E1F7F02128E7D7D447E1F7F02128E7D7D857E1F7F02128E7D7DC87E1F7F9E
:2057A00002128E7D7D1A7E1C7F02128E7D7DF87E1F7F02128E7D7D487E207F02128E7D7DCD
:2057C000B77E1B7F02128E7D7D567E207F02128E7D7D7F7E207F02128E7D7DB77E1B7F0246
:2057E000128E7D7DB87E207F02128E7D784A7600784AE624B0400CE4FD7C2D126E99784AB6
:205800000680EDC2981270C1EC90F90CF080002290FA47E0146003025D7B90F90CE0120DCF
:20582000775840315AA3325ADD335B66365C00375CA6385CF1395CF93F5D006100005D781E
:2058400090F915E0B44C028003025A947DDE7E207F02128E7D7D0A7E217F02128E7D744442
:2058600090F916F07D2A7E217F02128E7D1270C1EC90F90CF0B43102800302596790FA0E3D
:20588000E0640270030259677D5E7E217F02128E7D126FD9789E1213CBE4FB7A0679417884
:2058A000907403120472700B798F78B074071204727015EC4D4E4F600C7D767E217F0212BF
:2058C0008E7D1270C1025967789E121405E4FA790378E81202EE120B0C7A187B56785A79E4
:2058E00096120877120AB4789E1213CB0876007C0112482D78961213CB7C0112482D78A20D
:2059000006789A1213CB78961214117405120472700778A2E624F650D6C3789979A1E79617
:20592000FC1819E796FD30E706C3E49CFCE49DC3FDEC9404ED6480948050077C011234564A
:2059400080251818E6084608460846700E7D8D7E217F02128E7D1270C1800C7D9E7E217FD5
:2059600002128E7D1270C190F90CE0B432028003025A5F90FA15E064027003025A5F7D5E3C
:205980007E217F02128E7D126FD9789E1213CBE4FB7A06794178907403120472700B798FC7
:2059A00078B074071204727015EC4D4E4F600C7D767E217F02128E7D1270C1025A5D789EB3
:2059C000121405E4FA790378E81202EE120B0C7A187B56785A7996120877120AB4789E12EA
:2059E00013CB0876007C0212482D78961213CB7C0212482D78A206789A1213CB78961214ED
:205A0000117405120472700778A2E624F650D6C3789979A1E796FC1819E796FD30E706C3CB
:205A2000E49CFCE49DC3FDEC9404ED6480948050077C0212345680251818E6084608460870
:205A400046700E7D8D7E217F02128E7D1270C1800C7D9E7E217F02128E7D1270C18033908E
:205A6000F90CE0B4310890FA0EE06402600E90F90CE0B4321D90FA15E0B4021690F90CE0D0
:205A8000783F760008F67DB27E217F02128E7D1270C1800C7DE37E217F02128E7D1270C1C0
:205AA000025D787D0D7E227F02128E7D1270C1EC90F90CF0B431077C0112681D801CB43211
:205AC000077C0212681D801264616004ECB4410A7C0112681D7C0212681D025D7890F91566
:205AE000E0B44C737D527E227F02128E7D7D0A7E217F02128E7D744490F916F07D867E2298
:205B00007F02128E7D1270C1EC90F90CF0B4310F90FA0EE0640260077C01123FC68036ECC4
:205B2000B4320F90FA15E0640260077C02123FC6802390FA0EE06402600790FA15E0B40272
:205B4000147400783FF608ECF67DB27E217F02128E7D1270C1800C7DC17E227F02128E7D6F
:205B60001270C1025D787DF07E227F02128E7D789676007896E624CE4036E625E0242DF54F
:205B800082E434F9F583E0FDA3E07840F6ED18F67D087E237F02128E7D90F91BE078966635
:205BA00070097D0C7E237F02128E7D78960680C37D0F7E237F02128E7D789676007896E60A
:205BC00024CE4036E625E02491F582E434F9F583E0FDA3E07840F6ED18F67D087E237F020D
:205BE000128E7D90F91CE078966670097D0C7E237F02128E7D78960680C31270C1025D78DD
:205C000090F915E0B44C028003025C9790F9FBE0FDA3E0FCE4FB7A3C1201ECE87840F6E999
:205C200018F67D277E237F02128E7D7D5A7E237F02128E7D126FD978961213CBE4F9FAFB33
:205C4000780A7403120472703A7878740F1204727031ECFAEDFB783C12016D90F9FBE9F01E
:205C6000A3E8F0FEE9FF7C6D124E857896121405793F1213D77D757E237F02128E7D127055
:205C8000C18012EC4D4E4F600C7D987E237F02128E7D1270C1800C7DC17E227F02128E7DD0
:205CA0001270C1025D787DAB7E237F02128E7D1270C1EC90F90CF0646C6004ECB44C1B7400
:205CC0004C90F915F090F9F9E4F0A3F078A6C654FDF6FC7D07126EB9801464616004ECB4C0
:205CE000410C744190F915F0744590F916F0025D78740290FA47F0807F7C041250CA80781B
:205D000090F925121460783F1213CB7DDB7E237F02128E7D90F9FD121460783F1213CB7DE1
:205D2000FA7E237F02128E7D90FA05121460783F1213CB7D197E247F02128E7D90F92912D4
:205D40001460783F1213CB7D387E247F02128E7D90FA01121460783F1213CB7D577E247F86
:205D600002128E7D90FA09121460783F1213CB7D767E247F02128E7D0261CFE0B4020280C7
:205D8000030261CC90F90CE0120D775DB2315DF8325F2A335F39345F903560F936614038EB
:205DA00061C2395DAA3F000061CA7C051250CA0261CA90F915E0B44C307D957E247F021247
:205DC0008E7D1270C1EC90F90CF064796004ECB459157DFF7C6B124DBC7DCC7E247F0212B9
:205DE0008E7D7C0112F79B800C7DC17E227F02128E7D1270C10261CA789A76000876007D7C
:205E0000E57E247F02128E7D1270C1EC90F90CF0B431028003025E9D7D207E257F02128EE1
:205E20007D1270C1EC90F90CF064756004ECB4550A7899760108087601801264446004EC5C
:205E4000B4640A78997600087601087601789BE61470477D4C7E257F02128E7D126FD978FB
:205E600096EDF608ECF6789AE6793FF718E6FF7E011264BB7898ECF67C01126BF77898E692
:205E800014700E7D657E257F02128E7D1270C180097D807E257F02128E7D025F27B43202D3
:205EA0008003025F277D207E257F02128E7D1270C1EC90F90CF064756004ECB4550A7899F8
:205EC000760108087601801264446004ECB4640A78997600087601087601789BE6147047CF
:205EE0007D4C7E257F02128E7D126FD97896EDF608ECF6789AE6793FF718E6FF7E021264C9
:205F0000BB7898ECF67C02126BF77898E614700E7D657E257F02128E7D1270C180097D806E
:205F20007E257F02128E7D0261CA7DA67E257F02128E7D1270C10261CA90F915E0B44C4160
:205F40007DCE7E257F02128E7D786E76010876F90876F57DFB7E257F02128EB178967600FD
:205F60007896E624FD4018E624F5F582E434F9F583E0FDE62468FC124DBC78960680E1805A
:205F80000C7DC17E227F02128E7D1270C10261CA7D2A7E217F02128E7D1270C1EC90F90C61
:205FA000F0B43102800302604D7DFF7E257F02128E7D126FD978961213CBE4FB7A067941AA
:205FC00078907403120472700B798F78B074071204727014EC4D4E4F600C7D767E217F0233
:205FE000128E7D1270C1806290F912E0540F4440F0FC7D05126EB9126E2E7896121405E48B
:20600000FAFB790378E81202EE120B0C7A187B56785A7996120877120AB4789A1213CB7865
:206020003D7601126C257D1B7E267F02128E7D7D017C0112312B1270C1EC90F90CF064713D
:206040006008EC64516003EC70E50260F6B4320280030260F67DFF7E257F02128E7D126F3A
:20606000D978961213CBE4FB7A06794178907403120472700B798F78B074071204727014F7
:20608000EC4D4E4F600C7D767E217F02128E7D1270C1806290F912E0540F4440F0FC7D0599
:2060A000126EB9126E2E7896121405E4FAFB790378E81202EE120B0C7A187B56785A79969C
:2060C000120877120AB4789A1213CB783D7601126C257D1B7E267F02128E7D7D017C0212A6
:2060E000312B1270C1EC90F90CF064716008EC64516003EC70E50261CA90F915E0B44C3132
:206100007D387E267F02128E7D1270C1EC90F90CF064646004ECB44408744490F916F080F5
:206120000E64656004ECB44506744590F916F0800C7DC17E227F02128E7D1270C10261CA79
:2061400090F915E0B44C6D7D637E267F02128E7DE4786EF608F60876967D757E267F021237
:206160008EB17D527E8F7F027996E4FAFB75F003120DA04B70307D797E267F02128E7D7DD4
:206180008B7E267F02128E7D1270C1EC90F90CF0B431057C0112279690F90CE0B432057C6C
:2061A00002122796800C7DC57E267F02128E7D1270C1800C7DC17E227F02128E7D1270C170
:2061C0008008740190FA47F080008003B40300227C00124D07EC90FA0FF064596040744EAF
:2061E000F0742090FA0DF0740390FA0EF090FA10E4F0A3F0A3F0A3F090F925F0A3F0A3F0AA
:20620000A3F090F911E04401F0FC7D06126EB978A6C654FEF6FC7D07126EB90262F17C705E
:20622000124E41E4FEFF90F9FD12143F7C72124E41E4FEFF90FA0512143F7C03124D07ECBC
:2062400090FA0DF07C06124D07EC90FA0EF07C01124E41E4FEFF90F92512143F90FA0DE0D2
:206260006450600690FA0EE0600D90FA10E4F0A3F0A3F0A3F080347C04124E41E4FEFFF84A
:20628000F9FB04FA12052090F91D12143F120B0C7A187B56785A79961208777A7A7B441207
:2062A000086F120AB490FA1012143F90FA0DE0B4500C78A6C654FDF6FC7D07126EB990FAA3
:2062C0000EE0601990F911E04401F0FC7D06126EB978A6C654FEF6FC7D07126EB990FA0D74
:2062E000E0B4740D90F911E04402F0FC7D06126EB97C0A124D07EC90FA16F06459604074E8
:206300004EF0742090FA14F0740390FA15F090FA17E4F0A3F0A3F0A3F090F929F0A3F0A311
:20632000F0A3F090F911E04404F0FC7D06126EB978A6C654FEF6FC7D07126EB90264127C97
:2063400074124E41E4FEFF90FA0112143F7C76124E41E4FEFF90FA0912143F7C0D124D07FC
:20636000EC90FA14F07C10124D07EC90FA15F07C0B124E41E4FEFF90F92912143F90FA1478
:20638000E06450600690FA15E0600D90FA17E4F0A3F0A3F0A3F080347C0E124E41E4FEFF29
:2063A000F8F9FB04FA12052090F92112143F120B0C7A187B56785A79961208777A7A7B44FC
:2063C00012086F120AB490FA1712143F90FA14E0B4500C78A6C654FDF6FC7D07126EB9905C
:2063E000FA15E0601990F911E04404F0FC7D06126EB978A6C654FEF6FC7D07126EB990FA5C
:2064000014E0B4740D90F911E04408F0FC7D06126EB9742090FA1BF0E490FA1CF0744E90F0
:20642000FA1DF090FA1EE4F0A3F0A3F0A3F0742090FA22F0E490FA23F0744E90FA24F0907F
:20644000FA25E4F0A3F0A3F0A3F0742090FA29F0E490FA2AF0744E90FA2BF090FA2CE4F0E0
:20646000A3F0A3F0A3F0742090FA30F0E490FA31F0744E90FA32F090FA33E4F0A3F0A3F071
:20648000A3F0742090FA37F0E490FA38F0744E90FA39F090FA3AE4F0A3F0A3F0A3F0742034
:2064A00090FA3EF0E490FA3FF0744E90FA40F090FA41E4F0A3F0A3F0A3F0227835E4F60802
:2064C00004F608E4F60804F6783EEFF618EEF61818EDF608ECF6EF7013783FE614700DECBE
:2064E0002414FCE43D783BF608CCF6CCD3783CE6940018E6648094805003026729783EE690
:20650000702E18E6142445F582E434FAF583E014F0E6142445F582E434FAF583E033500EA8
:20652000E6142445F582E434FAF5837403F0802B18E6142445F582E434FAF583E004F0E6AF
:20654000142445F582E434FAF583E0B4040DE6142445F582E434FAF583E4F0E6142445F588
:2065600082E434FAF583E024A8F8E6FC783DE6FD126EB9783DE6FC12672EBC00067837E425
:20658000F608F6783DE61475F007A4240DF582E434FAF583E06450601108E6700D7837E611
:2065A00008467006740190FA48F090FA48E0147019783EE61470137838E6141846700B904B
:2065C000F917E07005E490FA48F090FA48E07027783EE614702190F917E0701B7837E6087E
:2065E000467014783DE61475F007A4240DF582E434FAF5837450F0783DE61475F007A42449
:206600000DF582E434FAF583E0B450227838E6141846701A90F917E07014783DE61475F0BC
:2066200007A4240DF582E434FAF5837420F0783DE61475F007A4240DF582E434FAF583E028
:20664000B4500A08E6700690F917E0600790F91AE01470077837E4F60804F690FA48E01482
:206660007013783EE614700D90F917E070077837E4F60804F6C37836E6941418E694005007
:2066800036D3783CE6940118E6648094804028E4FEFF7D017C907835E6FB08E6FA1201EC84
:2066A000E8D39EE99F40070EBE00010F80E47839EFF608EEF6801AE4FEFFC3EE9428EF9485
:2066C0000050070EBE00010F80F07839EFF608EEF6783606E61870010608E624FFFC18E661
:2066E00034FF783CFDEC667003ED1866701B783EE6701608E6147011783BE4F608761478BF
:2067000035F60804F6783E76017836E624FFFC18E634FF783CFDECC396ED1896500B78389F
:20672000E614184670030264FD7838E6FC22782C7601782FECF6B401028003D3400BE5DBBB
:2067400020E404782C76008039B402028003D3400BE5DB20E504782C76008026B403028043
:2067600003D3400BE5DB20E604782C76008013B404028003D3400BE5DB20E704782C760041
:206780008000782CE67D00FC90FA4AE06C700A90FA49E06D700302681A7C01ECF608E4F684
:2067A00008F618E6FF08E6FEC3EE9450EF94C350070EBE00010F80F0782DEFF608EEF608F6
:2067C000E6B401028003D3400BE5DB20E404782C76008039B402028003D3400BE5DB20E5C2
:2067E00004782C76008026B403028003D3400BE5DB20E604782C76008013B404028003D3F4
:20680000400BE5DB20E704782C76008000782CE67D0090FA49CDF0A3CDF0E6FC227850EC19
:20682000F67400783FF608ECF67DDD7E267F02128E7D740190F917F0784A760108760008F7
:20684000E4F608F608F608F608E614701590F91D121460E4FB04FA78187986740312047246
:20686000701B7850E6B4023C90F921121460E4FB04FA78187986740B12047270277850E605
:206880001475F007A4240DF582E434FAF583E064506011783F76007850E6FE7F007D037C49
:2068A000E81264BB7850E6FC12672EBC000280030269E9784A7600C3784FE694E818E69423
:2068C000035024784AE6701F783F76007850E6FE7F01E4FD04FC1264BB784AECF6784F062E
:2068E000E61870010680D0784FE664E8700418E66403600302699F784AE6600302699F0877
:2069000008E4F608F6784AE6702BC3784DE6948818E69413501F783F76007850E6FE7F005E
:20692000E4FD04FC1264BB784AECF6784D06E61870010680D0783F76017850E6FE7F007D3B
:20694000077CD01264BBC3784DE6948818E694135048E4F608F6784AE614702BC3784DE64F
:20696000948818E69413501F783F76007850E6FE7F01E4FD04FC1264BB784AECF6784D060D
:20698000E61870010680CF784DE66488700418E664137004784B76018003187601804878B3
:2069A0004CE4F608F6784AE614702BC3784DE6948818E69413501F783F76007850E6FE7F66
:2069C00001E4FD04FC1264BB784AECF6784D06E61870010680CF784DE66488700418E66404
:2069E000137004784B76018048784CE4F608F6784AE614702BC3784DE6948818E69413509C
:206A00001F783F76007850E6FE7F01E4FD04FC1264BB784AECF6784D06E61870010680CFB9
:206A2000784DE66488700418E664137004784B76017850E6FC126BF7784BE66003026B2869
:206A40007850E614706A745090FA0DF0FD7C03124DBC7D007C06124DBCE490FA0EF0FFFE35
:206A60007C04124E8590FA10E4F0A3F0A3F0A3F090F911E054FDF0FC7D06126EB990F9117D
:206A8000E054FEF0FC7D06126EB978A6C654FDF6FC7D07126EB990FA0EE0701290FA15E0BF
:206AA000700C78A6C64401F6FC7D07126EB9806CE6B40268745090FA14F0FD7C0D124DBC9F
:206AC0007D007C10124DBCE490FA15F0FFFE7C0E124E8590FA17E4F0A3F0A3F0A3F090F9FC
:206AE00011E054F7F0FC7D06126EB990F911E054FBF0FC7D06126EB978A6C654FDF6FC7D9D
:206B000007126EB990FA0EE0701290FA15E0700C78A6C64401F6FC7D07126EB9E490F917E4
:206B2000F00490F919F0FC227850E614705D740290F90FF0742090FA0DF0FD7C03124DBC72
:206B40007D027C06124DBC740290FA0EF0E4FEFF7C04124E8590FA10E4F0A3F0A3F0A3F0AE
:206B600090F911E054FDF0FC7D06126EB990F911E04401F0FC7D06126EB978A6E630E0091E
:206B800054FEFCF67D07126EB9805FE6B4025B740290F910F0742090FA14F0FD7C0D124D18
:206BA000BC7D027C10124DBC740290FA15F0E4FEFF7C0E124E8590FA17E4F0A3F0A3F0A360
:206BC000F090F911E04404F0FC7D06126EB990F911E054F7F0FC7D06126EB978A6E630E0DA
:206BE0000954FEFCF67D07126EB9E490F917F00490F919F07C00227835ECF61CEC2445F5EE
:206C000082E434FAF583E024A8F8E6441BFC7835E6FD026EB97C0112681D7C0212681DE4BD
:206C200090F918F02278391213CB120B0C7B4F7AC778CE79FF120877E4F87B4679807ABBB2
:206C40001209B7120AB478301213CB78061204C77833E6543F7F0008CDF6CD08CCF6CCFED0
:206C6000ED540FFDECF8EDF9E4FAFBC8C0E07836EFF608EEF6D0E0C87C081204FDE8782CA2
:206C80001213E37836E6FD08E6FCE4FEFF782C120571E4F8F9FB7A70120551782C1213CBAE
:206CA000783DE6147004C2EB8002C2EC783876007838E624E84031782C121405E4F8F9FBFC
:206CC0007A80120541E4F8F9FB7A807405120472A2E09200A2E092E9D2EA782C7C01120592
:206CE000A6C2EA78380680C8783DE6147004D2EB8002D2EC22782D1213CB08E6147004C235
:206D0000EB8002C2EC782C7600782CE624E8402F08121405E4F8F9FB7A80120541E4F8F90F
:206D2000FB7A807405120472A2E09200A2E092E9D2EA782D7C011205A6C2EA180680CA7825
:206D400031E6147004D2EB8002D2EC22782EEDF618ECF6147004C2EB8002C2EC1876007887
:206D60002CE624F840210808E654806480600274FF04A2E09200A2E092E9D2EAC625E0F66F
:206D8000C2EA18180680D808E6147004D2EB8002D2EC22782FEEF61818EDF608ECF6EE149A
:206DA0007004C2EB8002C2EC18187600782CE624F040267C0008E65480D3FDEC7005ED6418
:206DC000806001C392E99200D2EA08E625E0F618E633F6C2EA180680D3782FE6147008D22E
:206DE000EBC2EBD2EB8006D2ECC2ECD2EC22C2EA7D627C01126D4C7E017C017D40126D93CE
:206E000078317601E4FF7C3F7EB77DFF126CF57D627C02126D4C7E027C017D20126D937844
:206E2000317602E4FF7C307D917EF1026CF57E027D267C40126D9378317601E4FCFF7D05C8
:206E40007E70026CF57822764008760008760008ECF61818E6FD08E6FE1818E6FFEE24F98C
:206E6000400FEF7825566F70010DEFC313FF0E80EC7823EDF608EEF61818EFF6ED20E00842
:206E80007825C6547FF680067825C64480F63099FDC2997825E6F599227826EDF608ECF664
:206EA000640A4D70057C0D126E457827E6FC126E457826E6FD08E6FC227833ECF67831F655
:206EC000E418F67834EDF67830E6FF08E6FE0876007832E624F84021EE25E0CF33CFFEC2A9
:206EE00092D291EFFD7C005401D394004004D2918002C291D2920680D81818EFF608EEF63A
:206F00007834E6FC026F26D291D292C293C2FE7F00EF24F84007C2FFD2FF0F80F4782CEFF7
:206F2000F6D293C29322782CE4F608F60808ECF61470067C01ECF68037ECB402057402F65E
:206F4000802EB403057404F68026B404057408F6801EB405057410F68016B406057420F6CF
:206F6000800EB407057440F68006B408037480F67D00782CCDF6CD08F6FC087600782EE635
:206F800024F8401FEC25E0CD33CDFCC2FFEDFF7E005401D394004004D2FE8002C2FED2FFAE
:206FA0000680DA1818EDF608ECF6D293C293C2FE7F00EF24F84007C2FFD2FF0F80F4782E6E
:206FC000EFF6D293C293227DF17E267F02128E7D7DF67E267F02028E7DE47878F608F608CB
:206FE000767108087600E4786EF608F60876717DFA7E267F02128EB1E47878F608F6087644
:207000007108760078781213F3121011601F121011645A6006121011B47A06787C7601801E
:207020000C0DED70010E78781213B980D7787CE67033E47878F608F608767178781213F36A
:20704000121011602012101124D0500712101124C65006787B7601800C0DED70010E78782D
:207060001213B980D6787CE6700E18E61470097DFE7E267F02128E7D787BE614700708E6EA
:207080007003026FE6787CE6147006E4FCFDFEFF227D71E4FEFF0271C975AADC43BA03437D
:2070A0008780D2DFC29FD29EC29DD29CC298C299D288C289D2A8C2C8C2C9C2ADD2CFD2AF00
:2070C0002290F9F9E0FDA3E07831CDF6CD08F6782C7680087600783076007832E6240AFC85
:2070E00018E63400FD90F9FAE0D39C90F9F9E09D4005D2981876013098E07830E6703BC2AF
:20710000981818A69918E6FD18E6FF7E00EE24F8400FEF782E566F70010DEFC313FF0E806F
:20712000EC782DEDF60808EEF6782CEFF6ED20E006E599547FFC227C0022C2987C0022C0A6
:20714000E0C082C083740190F918F01490F90FF090F910F0D083D082D0E032C0E0C082C076
:2071600083C0D0E8C0E0ECC0E0EDC0E0C2C8C2C678A706E6B4071090F9FAE004F090F9F99A
:207180007003E004F0760090F915E0B44C2790F9F9E0FDA3E0FC90F9FCE0D39C90F9FBE077
:2071A0009D5012744190F915F0744590F916F0740190FA47F0D2C8D0E0FDD0E0FCD0E0F874
:2071C000D0D0D083D082D0E03278321213B978321213F3121011908F679330E30C0DED7069
:2071E000010E78321213B980E5121011B42D130DED70010E78321213B9783074FFF608F65C
:2072000080177830E4F60804F6121011B42B0A0DED70010E78321213B9782CE4F608F608B2
:20722000F608F678321213F3121011908F679330E23812134B78321213B9121007FCE4FD04
:20724000FEFF121362782C121405E4F9FAFB780A1202EE1213A712052078D074FFF9FAFBD9
:20726000120520782C1213CB80B97830E6FD08E6FCED3395E0FEFF782C1214110202EE78BE
:207280002CE4F608F6081213B9782E1213F3121096121007908F679330E26678311213FC0A
:2072A0001210374D605B782E1213F3121096E9FC7401120297ECF91210077D00FC782CE6E1
:2072C000FF08E6FEE4FB7A0A120162EC28FCED39FDEC24D0782DF6ED34FF18F6E6FD08E63E
:2072E000D394E8ED64809483400A7F037EE818EFF608EEF678311213F374FFFB1202AE80CB
:2073000088782CE6FD08E6FC22782D1213B9121096121007782CF6782CE6908F679330E39E
:2073200014081213F37401120297121096121007782CF680E2E6FC22782CECF608EDF6ECBB
:20734000908F679330E105EC545F8001EC18F624BF500BE624A54006C624C9F6800EE69301
:2073600030E206C624D0F680037C6422EDD39650037C6422E6FC2278311213B91273097884
:2073800030ECF6642B6004ECB42D3278371213F312104B4B602774FFFB1202AEECB42D0ADC
:2073A00078341213F3740112124478311213F374011202971210961210077830F67830E63E
:2073C000FC22782DEDF618ECF6782E1213F3121011782C66700408E6FC220DED70010E1207
:2073E0001011782EFC1213B9EC6006121011B45DD8782DE6600274FF04FC22782C76410899
:20740000762008E4F608F608763F08768008F608F608EDF608ECF67834E608466035E630DF
:20742000E009782C12140508120C447D017834E608FCE6CCA2E713CC13CCDDF8CCF6CC18A2
:20744000F64C600D782C1214051206F6782C1213CB80C47830021405121096785A1213B99D
:20746000784C1213C27840E4F608F6785D1213F3121096121007783BF67003027ED3908F75
:20748000679330E32D785A1213F3121096121007908F679330E30BE4FB049000011202BD6B
:2074A00080E3785D1213F3E4FB049000011202BD80B9121096121007B4250D1210969000EF
:2074C0000112100C646E6010785A1213F31210961210077003027E9E783BE66425603078B5
:2074E0005D1213F3E4FB049000011202BD785A1213F3127309EC783B666003027ED3785ACD
:207500001213F3E4FB049000011202BD02746B087600785D1213F3740112029712109612D8
:207520001007783BF6B42A157401120297121096121007783BF618C654FEF6800518C64421
:2075400001F608E6908F679330E2297842760208E4F67831F608F608764212727F7844EDD5
:20756000F608ECF6785D1213F3121096121007783BF680077844760208E4F68006783AC619
:2075800054F3F6783BE6646C6004E6B44C1518C64408F67401120297121096121007783B12
:2075A000F6801DB46815800518C64404F67401120297121096121007783BF618C654F7F69D
:2075C000E4FB049000011202BD783BE6120D777E842576094576094779D6587C125B7D3544
:2075E000637A89647609657609667609677A896879DF697E4A6E79CC6F7A7A707DBB737A73
:20760000897579D67800007EC8E47837F608F60876447834F608F608763C785A1213F312C0
:207620007377783BECF67844E6FD08E67843F6ED18F6784FE4F608F6785814F608F678445F
:20764000E608466023783BE6B4301D7845E61618700116785A1213F37401120297121096BF
:20766000121007783BF680D67844E6084670030276F8783BE6908F679330E27C785906E612
:2076800018700106E6FD08E664264D7003027E9E8021785906E618700106E6FD08E6FC78F0
:2076A0003AE654087E267F00EC6E7002ED6F7003027E9E7845E61618700116783BE624D08D
:2076C000FCE434FFFD120AFB121362784F1214057A207B411206F01213A71209B7784F1235
:2076E00013CB785A1213F37401120297121096121007783BF6027668783BE6B42E02800338
:207700000277857844E60846607B7845E616187001167843E616187001167853763F0876F4
:207720008008E4F608F67844E608466058785A1213F37401120297121096121007783BF6AD
:20774000908F679330E23E7845E61618700116783BE624D0FCE434FFFD120AFB12136278B5
:20776000537CCD7DCC7ECC7F3D120C441213A71206FE784F120C3F600A7853E608467003DA
:20778000027E9E80A17842E6FD08E67845667003ED18667003027E9E7844E6FD08E6FC788C
:2077A00045E61618700116EC4D700302790D783BE6FF908F679330E005EF44208001EFB478
:2077C0006502800302790D785A1213F3740112029778577600E47837F608F60876447834F3
:2077E000F608F6087657127377EC908F679320E203027E9EE47831F608F6087644785A1275
:2078000013F312727F7842EDF608ECF67857E66050784F121405081213CBD37843E694265B
:2078200018E6648094804003027E9E7842E6FD08E6FC1273FB784F120C497853E60846605D
:2078400007EE4F7003027E9E8014783AE620E30E7A807B00740B120BA97003027E9E027950
:207860000D7853747FF608F60874FFF608F67846E4F6087626802C783AE630E30A747FFE4C
:20788000FF74FFFCFD8008747FFEFF74FFFCFD78531213CB783AE654087C260D7846EDF69A
:2078A00008ECF678437959E726FC1819E7367847FDECD39618E66480CD64809D4003027EF6
:2078C0009E784309E726FC1819E7367847FDEC667003ED18667027C378597947E796FC1887
:2078E00019E796FD1273FB7853121411120877784F121411740B120BB37003027E9E78424A
:20790000E6FD08E6FC1273FB784F120C44783AE620E0030279C9807330E3380808E6600F6F
:20792000784F121405EE4F6004EF6480FF8005784F12140578601213FC121362121091ED4B
:20794000FC74031202CFECFD1210961213951212BC80360808E6600F784F121405EE4F60EC
:2079600004EF6480FF8005784F12140578601213FC121362121091EDFC74031202CFECFD5B
:207980001210961213951212BC80360808E6600F784F121405EE4F6004EF6480FF80057818
:2079A0004F12140578601213FC121362121091EDFC74031202CFECFD121096121395121258
:2079C000BC784106E61870010602746B7846E4F6087608027A907846E4F608761080077887
:2079E00046E4F608760A7837F608F60876447834F608F608763C785A1213F3127377783B87
:207A0000ECF6B430737844E60846606C785A1213F312109690000112100C908F679330E0E7
:207A20000D12109690000112100C4420800912109690000112100CB47830D37845E69401F7
:207A400018E66480948040227402120297121096121007783BF67845E624FEF618E634FF37
:207A6000F67846E4F6087610800E7847E6640A18467005E4F608760880337846E4F608764D
:207A800010783AC64408F680077846E4F608760AE47837F608F60876447834F608F608760E
:207AA0003C785A1213F3127377783BECF67844E60846600F7847E6FD783BE6FC127338ECD0
:207AC000B46403027E9E7848E4F608F608F608F67847E6FD785A1213FCEDC0E012109112F2
:207AE0001011FCD0E0FD1273387D007842EDF608ECF66464604C08E6FD08E6FC7845E616F9
:207B000018700116EC4D603A7846E6FD08E6FCED3395E0FEFF081214111202EE7842E6FBFA
:207B200008E6F8EBF93395E0FBFA12052078481213CB785A1213F3E4FB049000011202BDC8
:207B4000808E783AE620E003027C0F0808E66005784812058B783AE630E324784812140578
:207B600078601213FC121362121091EDFC74031202CFECFD1210961213951212BC802A7832
:207B80004AE6FD08E6FC78601213FCEDC0E0ECC0E0121091EDFC74031202CFECFD12109625
:207BA000D0E0FDD0E0CD121272805C783AE630E22C784AE6FD08E6FC78601213FCEDC0E03E
:207BC000ECC0E0121091EDFC74031202CFECFD121096D0E0FDD0E0CD121272802A784AE670
:207BE000FD08E6FC78601213FCEDC0E0ECC0E0121091EDFC74031202CFECFD121096D0E045
:207C0000FDD0E0CD121272784106E61870010602746B783AE630E01978601213F3121096D6
:207C2000E9FC7403120297ECF9121091783D1213B9785D1213F3121096121007783BF6B4E7
:207C40005E130876007401120297121096121007783BF680030876017003027D32783AC6ED
:207C60004402F67844E6FD08E6FC7845E61618700116EC4D607B785A1213F312109612100F
:207C800007606E785D1213F3121096782E1213C2783CE6FD785A1213FCEDC0E01210911201
:207CA0001011FCD0E0FD1273C2EC6040783AE630E11130E008784106E618700106783AC6A9
:207CC00054FDF6E630E015785A1213F3121096121007FC783D121317EC12123D785A121356
:207CE000F3E4FB049000011202BD80028003027C63783AE620E11230E00F783D1213F3E4EB
:207D0000121244783AC64402F6C654FEF6785D1213F37401120297121096121007783BF6A2
:207D20006010B45D0BE4FB049000011202BD800280DB027E30783AE630E01978601213F334
:207D4000121096E9FC7403120297ECF9121091783D1213B97845E6700418E66402700778CF
:207D600044E4F60804F67844E6FD08E6FC7845E61618700116EC4D602E785A1213F312102F
:207D8000961210076021783AE630E010121096121007FC783D121317EC12123DE4FB04905D
:207DA00000011202BD80BF783AE654017D00FC7841E62CF618E63DF602746B783AE630E0D1
:207DC0001978601213F3121096E9FC7403120297ECF9121091783D1213B9785A1213F312B4
:207DE00073097844E6FD08E6FC7845E61618700116EC4D603B785A1213F312109612100787
:207E0000602E121096121007908F679320E321783AE630E010121096121007FC783D121347
:207E200017EC12123DE4FB049000011202BD80B2783AE630E011784106E618700106783DC5
:207E40001213F3E412124402746B785A1213F3900001121046C3784E96FA18EB96FB786075
:207E60001213F3EBC0E0EAC0E0121096E9FC7403120297ECF9121091D0E0FBD0E0CB121234
:207E80007C02746B785A1213F3121096E9FC7401120297ECF9121007B4250302746B785A41
:207EA0001213F3121096121007701D785D1213F3121096121007908F679330E30BE4FB0454
:207EC0009000011202BD80E37840E6FD08E6FC2202746B7840E6FD08E6FC2290F802E4F050
:207EE000A3F0782C1213B9782C12132612101190F80EF06425602FE0700990F802E0FDA34A
:207F0000E0FC22FC78311213F3782F868308868212142712143490F803E004F090F80270E6
:207F200003E004F080C1782C1213F3121011B4252E0DED70010E782C1213B978311213F377
:207F4000782F86830886821214277C2512143490F803E004F090F8027003E004F080887D64
:207F6000217EF87F0190F81A12143690F8171214367D1A7E270F90F81D121436E4A3F0909E
:207F8000F80CF090F809F090F808F0782C1213F3121011B42B03B34011C3B420028003D328
:207FA000401690F808E06002803E782C1213F312101190F808F08030B42D028003D340083B
:207FC00090F809E004F08020B423028003D3400890F80CE004F08010B430028003D34006AB
:207FE00090F820E004F0800A782E06E6187001068099782C1213F3121011B42A3E78341278
:2080000013F3121096E9FC7402120297ECF912103790F800CDF0A3CDF0ED335014C3E0FC96
:20802000E49CF090F800E0FCE49CF090F809E004F0782E06E618700106804D90F800E4F04D
:20804000A3F0782C1213F312101124D0503A12101124C6403390F800E0A3E0782C121326B6
:2080600012101124D0FCE434FFFD90F800E0FFA3E0FEE4FB7A0A120162EC28FCED3990F84B
:2080800000F0A3CCF0CC80BA90F809E06005E490F820F0782C1213F3121011B42E028003E3
:2080A00002812A0DED70010E121011782CFC1213B9ECB42A2678341213F3121096E9FC7424
:2080C00002120297ECF912103790F804CDF0A3CDF0782E06E618700106804D90F804E4F0BE
:2080E000A3F0782C1213F312101124D0503A12101124C6403390F804E0A3E0782C12132612
:2081000012101124D0FCE434FFFD90F804E0FFA3E0FEE4FB7A0A120162EC28FCED3990F8A6
:2081200004F0A3CCF0CC80BA800890F80474FFF0A3F0E490F80BF090F80AF0782C1213F337
:20814000121011B44C03B34009C3B46C028003D3401090F80AE004F0782E06E618700106DB
:208160008016B468028003D3400E90F80BE004F0782E06E618700106782C121326121011FD
:2081800090F80EF0120D778C9A00865845863047835658826B6384426486586586536686CA
:2081A000306784426981BB6E832F6F835670829773835675834A7800008CA28002807E8098
:2081C0004990F80BE06002801090F80AE06002803F806A90F80BE0602D90F802E0FDA3E08A
:2081E000FC78341213FCEDC0E0ECC0E0121091EDFC74031202CFECFD121096D0E0FDD0E0A9
:20820000CD12127280028035805E90F80AE0602D90F802E0FDA3E0FCED3395E0FEFF7834C3
:208220001213FC121362121091EDFC74031202CFECFD1210961213951212BC802B90F80230
:20824000E0FDA3E0FC78341213FCEDC0E0ECC0E0121091EDFC74031202CFECFD121096D075
:20826000E0FDD0E0CD121272027EE778341213F3121096E9FC7402120297ECF9900001129D
:20828000100C90F821F090F81CE004F090F81B7003E004F0028CB978341213F3121096E91B
:2082A000FC7403120297ECF912109190F817121436ED4E700C7D2B7E277F0290F8171214C3
:2082C0003690F804E03350077427F0A37410F090F806E4F0A3F090F817121335121011604F
:2082E0002B90F806E0FDA3E0FC90F805E0D39C90F804E06480CD6480CD9D401090F807E063
:2083000004F090F8067003E004F080CA90F81712148EA3A312143690F806E0FBA3E0FA90DF
:20832000F819C3E09AF090F818E09BF0028CB990F80CE0601590F804E0FDA3E04D700BE030
:2083400004F090F8047003E004F07D3A7E277F0290F81D12143690F80EE0B4701F78341201
:2083600013F3121096E9FC7403120297ECF9121091EDFCEEFDEFFE7F00028409801A78348B
:208380001213F3121096E9FC7402120297ECF9121037FCE4FEFF807190F80AE06016783467
:2083A0001213F3121096E9FC7404120297ECF912112F801878341213F3121096E9FC74023F
:2083C000120297ECF9121037FCE4FEFF803B90F80BE0601A78341213F3121096E9FC740258
:2083E000120297ECF9121037FCE4FEFF801B78341213F3121096E9FC7402120297ECF912A3
:208400001037FCED3395E0FEFF90F80F12143F90F80EE0FFB46F08E4F9FAFB78088015FC08
:208420006475600274FF046004740A80027410F8E4F9FAFB90F81312144BE990F808F00261
:208440008511802478341213F3121096E9FC7404120297ECF912112F90F80F12143FEF300C
:20846000E7030284F502850490F80AE0601678341213F3121096E9FC7404120297ECF912A9
:20848000112F801B78341213F3121096E9FC7402120297ECF9121037FCED3395E0FEFF9023
:2084A000F80F12143FEF30E702804A805790F80BE0601D78341213F3121096E9FC740212CE
:2084C0000297ECF9121037FCED3395E0FEFF801B78341213F3121096E9FC7402120297EC2E
:2084E000F9121037FCED3395E0FEFF90F80F12143FEF30E70F12045190F80F12143F742D87
:2085000090F808F090F813E4F0A3F0A3F0A3740AF07DA67EF87F0190F81A12143690F8177F
:2085200012143690F80F121460EC4D4E4F6002740190F80DF090F804E0FDA3E04D70069051
:20854000F80DE0603F90F81D12145712137490F80F121460A312146C1204028C828D83D084
:20856000E0FDD0E0FED0E0FF121016FC90F81712148EEC12124490F81312146090F80F121C
:2085800006AB70C190F804E033502B90F820E0602590F808E0600274017D00FCC3E49CFCD3
:2085A000E49DFD90F801E02CFC90F800E03D90F804F0A3CCF0CC90F81BE0FDA3E0C390F812
:2085C00019FEE0CE9EFC90F818E0FEED9EFD90F805E0D39C90F804E06480CD6480CD9D40AF
:2085E0000D90F81712148E743012124480C890F80CE06039A3E06035A3E064786004E0B44B
:20860000580EE0FC90F81712148EEC1212448012B46F0F90F8171214571210116430600268
:20862000800090F81712148E7430121244028CB990F80EE024FEF090F806E4F0A304F09003
:20864000F804E0FDA3E04D700890F804E4F0A304F0800CE490F80EF090F806E4F0A3F09087
:20866000F804E0335006E4F0A37406F0803E90F80AE0601678341213F3121096E9FC740435
:20868000120297ECF912112F801478341213F3121096E9FC7404120297ECF912112F90F821
:2086A000A712143FEF30E7028020803278341213F3121096E9FC7404120297ECF912112F99
:2086C00090F8A712143FEF30E714EE4F6004EF6480FF90F8A712143F742D90F808F090F83C
:2086E00000E0FEA3E0FD90F819E02DF0FD90F818E03EF0FE90F817E0FF90F81A12143690C9
:20870000F8B4E4F0A3F090F8A71214607B2E7ADB79E678FF740F120BB3702179027A157B54
:208720005078F91206FE90F8A712143F90F8B5E024F6F090F8B4E034FFF080CA90F8A712DD
:2087400014607A807B3F740B120BA97020E4F8F97A207B411206FE90F8A712143F90F8B50A
:20876000E024FFF090F8B4E034FFF080CF90F8A712146079437B5178B77ABA7403120BB391
:20878000702179027A157B5078F912088390F8A712143F90F8B5E0240AF090F8B4E0340046
:2087A000F080CA90F8A71214607A207B417403120BA97020E4F8F97A207B4112088390F857
:2087C000A712143F90F8B5E004F090F8B47003E004F080CF90F806E0FDA3E04D606090F827
:2087E000B4E0FDA3E0FC90F805E0D39C90F804E06480CD6480CD9D4025C3EC94FC90F8B442
:20880000E06480947F4017E0FBA3E0FA90F805C3E09AF090F804E09BF0E490F80EF090F82F
:2088200005E024FFF090F804E034FFF090F80CE0600990F806E4F0A3F080037401F090F86F
:208840000EE0600A90F8B2E4F0A3F002891590F8B4E033400302890290F81A1213357430C0
:2088600012124490F804E0FDA3E090F8AECDF0A3CDF04D700690F80CE0600B90F81A1213E8
:2088800035742E12124490F8B0E4F0A3F090F8B1E024FFF090F8B0E034FFF0E0FDA3E0FC37
:2088A00090F8B5E0C39C90F8B4E06480CD6480CD9D502590F804E0FDA3E04D601B90F81A56
:2088C000121335743012124490F805E024FFF090F804E034FFF080B590F8AEE0F4FDA3E064
:2088E000F4FC90F8B5E0C39C90F8B4E06480CD6480CD9D5003028AD390F8B2E4F0A304F09A
:208900008013E0FDA3E0FCC3E49CFCE49DFD90F8B2F0A3ECF090F8B2E0FDA3E0FC90F805DF
:20892000E0C39C90F804E06480CD6480CD9D406D90F8A7121460120AB490F8AEEDF0A3ECB9
:20894000F0120AFB90F8A7120C03E4F8F97A207B411206FE12143F90F8AFE02430FC90F82B
:208960001A121335EC12124490F8B2E0FDA3E0FCE004F090F8B27003E004F0EC4D701B90F0
:20898000F804E0FDA3E04D700690F80CE0600B90F81A121335742E12124402891590F8A704
:2089A0001214607AA07B407403120BA96003028AD390F81A121457ED1D70011E90F8AB1260
:2089C0001436A3E4F0A304F090F8AB121457121011642E602090F8AFE0120119B43A0F7496
:2089E0003012124490F8AEE4F0A304F0800790F8AEE4F0A3F012135790F8AB121436EAFD28
:208A0000E9FC90F819E0C39C90F818E09D40B990F8AEE0FDA3E04D7003028AD390F80EE050
:208A2000606990F81A12145790F8AB12143690F8ACE0FDA3E0FC90F819E0C39C90F818E0CF
:208A40009D503890F8AB12145790FFFF121016B42E1690FFFE121016121244ED1D70011EBD
:208A600090F8AB1214368006121016121244ED1D70011E90F8AB12143680B390F8B5E004C5
:208A8000F090F8B47003E004F0803D90F81A12147890F8AB12143690F8ACE0FDA3E0FC90B7
:208AA000F819E0C39C90F818E09D501C90F8AB12145790FFFF121016121244ED1D70011E66
:208AC00090F8AB12143680CF90F817121457743112124490F806E0FDA3E04D602D90F81A25
:208AE00012145790FFFF121016B4300DED1D70011E90F81A12143680E4121016B42E0BED35
:208B00001D70011E90F81A12143690F80EE07003028C35FC90F81A121335EC12124490F82B
:208B2000B4E033501E90F81A121335742D12124490F8B5C3E0FCE49CF090F8B4E0FCE49C17
:208B4000F0800B90F81A121335742B12124490F81CE0240AF090F81BE03400F090F8AEE434
:208B6000F0A3F090F8AFE004F090F8AE7003E004F090F8B4E0FDA3E0FCE4FB7A0A1201C418
:208B8000E82430FC90F81A121335EC121244E4FB7A0A90F8B4E0F9A3E0F812019A90F8B471
:208BA000E9F0A3E8F04970BBC390F8AFE0940290F8AEE06480948040AAE0FDA3E0A3CDF0C5
:208BC000A3CDF0D390F8AFE0940090F8AEE064809480405390F81A12145790F8AFE0C3CD50
:208BE0009DFD90F8AEE0CE9EFE121011FC90F81A121457E0FBA3E0C390F8B1F9E0C999FA7E
:208C000090F8B0E0F9EB99FBEA24F5FAEB34FF8A82F583EC12124B90F8AFE024FFF090F818
:208C2000AEE034FFF0809C90F81CE024F6F090F81BE034FFF090F820E0605D90F808E0601E
:208C40000274017D00FCC3E49CFCE49DFD90F801E02CFC90F800E03D90F804F0A3CCF0CC8A
:208C600090F81BE0FDA3E0C390F819FEE0CE9EFC90F818E0FEED9EFD90F805E0D39C90F8DD
:208C800004E06480CD6480CD9D400D90F81712148E743012124480C8801F782EE616187034
:208CA00001167D4B7E277F0290F817121436ED2403FD50010EA312143690F81BE0FDA3E042
:208CC000C390F819FEE0CE9EFC90F818E0FEED9E90F804F0A3CCF0CC90F800FDE0FFA3E053
:208CE000FEEDFBECD39EFAEF6480CB64809B4005E4FEFF802990F808E0600274017D00FC8B
:208D0000C3E49CFCE49DFDEC2EFCED3FC3FD90F805E0FAEC9AFE90F804E0FAED9AFF90F835
:208D200006EFF0A3EEF0A3A3E0703A90F807E024FFF090F806E034FFF0E0FDA3E0ED33402A
:208D40002478311213F3782F86830886821214277C2012143490F803E004F090F8027003CF
:208D6000E004F080C690F808E06021FC78311213F3782F868308868212142712143490F83C
:208D800003E004F090F8027003E004F090F805E024FFF090F804E034FFF0E0FDA3E0ED339C
:208DA000402C90F817121335121011FC78311213F3782F868308868212142712143490F86F
:208DC00003E004F090F8027003E004F080BE90F809E0603A90F807E024FFF090F806E0347E
:208DE000FFF0E0FDA3E0ED33402478311213F3782F86830886821214277C2012143490F854
:208E000003E004F090F8027003E004F080C6027EE778341213B978391213B9124ADE7837FB
:208E2000EDF608ECF6640A4D6015EC047004ED04600DECFE7834121317EC12123D80DCEC0C
:208E4000047002ED04701A78341213FC783BE9667008EA18667003EB18667005E4FDFEFF43
:208E60002278341213F3E412124478390213F378291213B97828ECF67D00026E99783C12BA
:208E800013B9E47837F608F608763F7834F608F60876377831F608F608F6782F7614087623
:208EA000AD783C1213F3127EDB783AEDF608ECF622786B1213B97869E4F608F67863760161
:208EC0000876F80876007D007EF87F01128E11ED4E6076E47866F608F608766E78631213C7
:208EE000F31210116021E47860F608F6087666785DF608F608766B7D63FEFF127458786AE8
:208F0000E62CF618E63DF6786B1213F3121011602678631213F3121011701C786376010858
:208F200076F80876007D007EF87F01128E11ED4E7005E490F800F0786B1213F31210117077
:208F40009B7869E6FD08E6FC2274FFFCFD2258314B0044554B4500202000544600504600AB
:208F60002020004346000020202020202020202028282828282020202020202020202020E0
:208F8000202020202020208810101010101010101010101010101004040404040404040455
:208FA0000410101010101010414141414141010101010101010101010101010101010101A5
:208FC00001011010101010104242424242420202020202020202020202020202020202027F
:208FE00002021010101020FFFFFFFFFFFFFFFFFFFFFFFFFFFFFFFFFFFFFFFFFFFFFFFFFF26
:20900000FFFFFFFFFFFFFFFFFFFFFFFFFFFFFFFFFFFFFFFFFFFFFFFFFFFFFFFFFFFFFFFF70
:20902000FFFFFFFFFFFFFFFFFFFFFFFFFFFFFFFFFFFFFFFFFFFFFFFFFFFFFFFFFFFFFFFF50
:20904000FFFFFFFFFFFFFFFFFFFFFFFFFFFFFFFFFFFFFFFFFFFFFFFFFFFFFFFFFFFFFFFF30
:20906000FFFFFFFFFFFFFFFFFFFFFFFFFFFFFFFFFFFFFFFFFFFFFFFFFFFFFFFFFFFFFFFF10
:20F78000FFFFFFFFFFFFFFFFFFFFFFFFFFFFFFFFFFFFFFFFFFFFFFFFFFFFFFC2AFECA2E0A5
:20F7A00092978C21E4FEFFC3EE94E8EF940350070EBE00010F80F0782CEFF608EEF60200C5
:20F7C00000FFFFFFFFFFFFFFFFFFFFFFFFFFFFFFFFFFFFFFFFFFFFFFFFFFFFFFFFFFFFFF48
:20F7E000FFFFFFFFFFFFFFFFFFFFFFFFFFFFFFFFFFFFFFFFFFFFFFFFFFFFFFFFFFFFFFFF29
:20F80000FFFFFFFFFFFFFFFFFFFFFFFFFFFFFFFFFFFFFFFFFFFFFFFFFFFFFFFFFFFFFFFF08
:20F82000FFFFFFFFFFFFFFFFFFFFFFFFFFFFFFFFFFFFFFFFFFFFFFFFFFFFFFFFFFFFFFFFE8
:20F84000FFFFFFFFFFFFFFFFFFFFFFFFFFFFFFFFFFFFFFFFFFFFFFFFFFFFFFFFFFFFFFFFC8
:020000021000EC
:00000001FF
